:020000040800F2
:1000000000070020F102000839340008F13300082D
:1000100019340008F133000811340008F302000815
:10002000F3020008F3020008F30200082544000868
:10003000F3020008F3020008F3020008F3020008CC
:10004000F3020008F3020008F3020008F3020008BC
:10005000F3020008F3020008DD7C0008097D0008B7
:10006000357D0008617D00088D7D0008E9440008A9
:10007000114500083D450008694500089545000800
:10008000BD450008E9450008F3020008A133000857
:10009000C9330008B5330008DD330008B97D000816
:1000A000F3020008F3020008F3020008F30200085C
:1000B000F3020008F3020008F3020008F30200084C
:1000C000F3020008F3020008F3020008F30200083C
:1000D000F3020008F3020008F3020008F30200082C
:1000E0001D7E0008F3020008F3020008F302000876
:1000F000F3020008F3020008F302000815460008A6
:10010000F3020008F3020008A57E0008F3020008CD
:10011000F3020008F3020008F3020008F3020008EB
:10012000414600086946000895460008C146000897
:10013000ED460008F3020008F3020008F30200088D
:10014000F3020008F3020008F3020008F3020008BB
:1001500015470008414700086D470008F3020008F2
:10016000F3020008F3020008F3020008F30200089B
:10017000F3020008E5700008F3020008F30200082B
:10018000F3020008F3020008917E0008F302000861
:10019000F3020008F3020008F3020008F30200086B
:1001A000F3020008F3020008F3020008F30200085B
:1001B000F3020008F3020008F3020008F30200084B
:1001C000F3020008F3020008F3020008F30200083B
:1001D000F3020008D1700008F3020008F3020008DF
:1001E000F3020008F3020008F3020008F30200081B
:1001F000F3020008F3020008F3020008F30200080B
:10020000F3020008F3020008F3020008F3020008FA
:10021000F3020008F3020008F3020008F3020008EA
:10022000F3020008F3020008F3020008F3020008DA
:10023000F3020008F3020008F3020008F3020008CA
:10024000F3020008F3020008F3020008F3020008BA
:10025000F3020008F3020008F3020008F3020008AA
:10026000F3020008F3020008F3020008F30200089A
:10027000F3020008F3020008F3020008F30200088A
:10028000F3020008F3020008F3020008F30200087A
:10029000F3020008F3020008F3020008F30200086A
:1002A000F3020008F3020008F3020008F30200085A
:1002B000F3020008F3020008F3020008F30200084A
:1002C000F3020008F3020008F3020008F30200083A
:1002D000F3020008F3020008F3020008F30200082A
:1002E00021170008000000000000000000000000CE
:1002F00002E000F000F8FEE772B6374880F30888A5
:10030000364880F3098836483649086040F20000D4
:10031000CCF200004EF63471CEF200010860BFF35B
:100320004F8FBFF36F8F40F20000C0F2F0004EF627
:100330008851CEF200010860BFF34F8FBFF36F8F7B
:100340004FF00000E1EE100A4EF63C71CEF20001D3
:100350000860062080F31488BFF36F8F06F02EF933
:1003600007F076FA4FF055301F491B4A91423CBFC7
:1003700041F8040BFAE71D49184A91423CBF41F885
:10038000040BFAE71A491B4A1B4B9A423EBF51F82D
:10039000040B42F8040BF8E700201849184A914270
:1003A0003CBF41F8040BFAE706F046F907F0D4FA2F
:1003B000144C154DAC4203DA54F8041B8847F9E796
:1003C00000F042F8114C124DAC4203DA54F8041B11
:1003D0008847F9E706F02EB9000700200023002027
:1003E0000000000808ED00E00001002000070020E8
:1003F00060850008002300206C230020702300206B
:1004000030890020E0020008E4020008E40200084D
:10041000E40200082DE9F04F2DED108AC1F80CD050
:10042000D0F80CD0BDEC108ABDE8F08F002383F328
:1004300011882846A047002005F0E4FAFEE705F001
:100440005FFA00DFFEE70000F8B501F0E9F901F01E
:100450007FFB06F037F8074606F0A6F80546A8BB6E
:100460001F4B9F4232D001339F4232D027F0FF0210
:100470001C4B9A4230D12E4642F21074F8B200F072
:100480009BFF00F09FFF08B10024264601F0F0FD1D
:1004900020B10024032000F079F8264635B1124B34
:1004A0009F4203D0002406F077F82646002006F08D
:1004B00013F80EB100F080F801F0E8FA00F0B6FF92
:1004C000204600F037F900F077F8F9E72E460024CF
:1004D000D7E704460126D4E7064641F28834D0E740
:1004E000010007B0000008B0263A09B008B501F0D5
:1004F00063F9A0F120035842584108BD07B541F205
:100500001203022101A8ADF8043001F073F903B021
:100510005DF804FB38B5302383F31188174803686E
:100520000BB105F03BFB0023154A4FF47A711348D9
:1005300005F02AFB002383F31188124C236813B1C2
:100540002368013B2360636813B16368013B636008
:100550000D4D2B7833B963687BB9022001F008FA9E
:10056000322363602B78032B07D163682BB90220F9
:1005700001F0FEF94FF47A73636038BD70230020F8
:10058000150500089024002088230020084B1870CF
:1005900003280CD8DFE800F008050208022001F06B
:1005A000E5B9022001F0E0B9024B00225A60704721
:1005B0008823002090240020F8B501F059FD30B1C7
:1005C000544B03221A700022534B5A60F8BD534B10
:1005D000534A1C4619680131F8D004339342F9D1CB
:1005E0006268504B9A42F1D94F4B9B6803F100630C
:1005F00003F500339A42E9D205F0A2FF05F0B4FFFB
:10060000002001F027F90220FFF7C0FF474B00212F
:10061000D3F8E820C3F8E810D3F81021C3F810117C
:10062000D3F81021D3F8EC20C3F8EC10D3F8142140
:10063000C3F81411D3F81421D3F8F020C3F8F01044
:10064000D3F81821C3F81811D3F81821D3F8802053
:1006500042F00062C3F88020D3F8802022F00062CC
:10066000C3F88020D3F88020D3F8802042F00072B5
:10067000C3F88020D3F8802022F00072C3F88020D5
:10068000D3F8803072B64FF0E023C3F8084DD4E9B8
:100690000004BFF34F8FBFF36F8F254AC2F8841059
:1006A000BFF34F8F536923F480335361BFF34F8FF0
:1006B000D2F8803043F6E076C3F3C905C3F34E3376
:1006C0005B0103EA060C29464CEA81770139C2F83E
:1006D0007472F9D2203B13F1200FF2D1BFF34F8F88
:1006E000BFF36F8FBFF34F8FBFF36F8F536923F447
:1006F000003353610023C2F85032BFF34F8FBFF372
:100700006F8F302383F31188854680F30888204754
:100710005CE700BF8823002090240020000002082E
:1007200020000208FFFF01080023002000440258B7
:1007300000ED00E02DE9F04F93B0B74B2022FF21F0
:1007400000900AA89D6801F04BF9B44A1378A3B948
:100750000121B34811700360302383F311880368CB
:100760000BB105F01BFA0023AE4A4FF47A71AC4886
:1007700005F00AFA002383F31188009B13B1AA4BFA
:10078000009A1A60A94A1378032B03D00023137030
:10079000A54A53604FF0000A009CD3465646D14606
:1007A000012001F0E3F824B19F4B1B68002B00F0FF
:1007B0002C82002001F000F80390039B002B01DA4B
:1007C00000F088FE039B002BEDDB012001F0CCF84C
:1007D000039B213B1F2BE3D801A252F823F000BF5B
:1007E00061080008890800081D090008A107000821
:1007F000A1070008A1070008AF0900087F0B000847
:10080000990A0008FB0A0008230B0008490B00089E
:10081000A10700085B0B0008A1070008CD0B00082A
:1008200001090008A1070008110C00086D08000864
:1008300001090008A1070008FB0A0008A107000839
:10084000A1070008A1070008A1070008A1070008E8
:10085000A1070008A1070008A10700081D0900085A
:100860000220FFF743FE002840F0F981009B02219F
:1008700005A8BAF1000F08BF1C4641F21233ADF8CB
:10088000143000F0B7FF8BE74FF47A7000F094FF5C
:10089000071EEBDB0220FFF729FE0028E6D0013F10
:1008A000052F00F2DE81DFE807F0030A0D10133692
:1008B0000523042105A8059300F09CFF17E00421FF
:1008C0005548F9E704215A48F6E704215948F3E767
:1008D0004FF01C08404608F1040800F0BDFF042159
:1008E000059005A800F086FFB8F12C0FF2D1012089
:1008F0004FF0000900FA07F747EA0B0B5FFA8BFB92
:1009000001F0BAF826B10BF00B030B2B08BF002443
:10091000FFF7F4FD44E704214748CDE7002EA5D0BA
:100920000BF00B030B2BA1D10220FFF7DFFD0746D5
:1009300000289BD00120002600F08CFF0220FFF74A
:1009400025FE1FFA86F8404600F094FF0446B0B139
:10095000039940460136A1F140025142514100F055
:10096000A1FF0028EDD1BA46044641F2121302213C
:1009700005A83E46ADF8143000F03CFF10E72546D0
:100980000120FFF703FE244B9B68AB4207D92846A2
:1009900000F062FF013040F067810435F3E7002585
:1009A000224BBA463E461D701F4B5D60A8E7002EE5
:1009B0003FF45CAF0BF00B030B2B7FF457AF02201F
:1009C000FFF7E4FD322000F0F7FEB0F10008FFF67B
:1009D0004DAF18F003077FF449AF0F4A08EB05034A
:1009E000926893423FF642AFB8F5807F3FF73EAF43
:1009F000124BB845019323DD4FF47A7000F0DCFE12
:100A00000390039A002AFFF631AF039A0137019B46
:100A100003F8012BEDE700BF002300208C24002009
:100A20007023002015050008902400208823002052
:100A300004230020082300200C2300208C23002006
:100A4000C820FFF753FD074600283FF40FAF1F2DC6
:100A500011D8C5F120020AAB25F0030084494245B4
:100A6000184428BF4246019200F094FF019AFF21EA
:100A70007F4800F0B5FF4FEAA803C8F387027C491E
:100A80002846019300F0B4FF064600283FF46DAFFE
:100A9000019B05EB830533E70220FFF727FD0028C4
:100AA0003FF4E4AE00F010FF00283FF4DFAE002773
:100AB000B846704B9B68BB4218D91F2F11D80A9BB0
:100AC00001330ED027F0030312AA134453F8203C3D
:100AD00005934046042205A9043701F0B3FA804685
:100AE000E7E7384600F0B8FE0590F2E7CDF814804D
:100AF000042105A800F07EFE02E70023642104A87B
:100B0000049300F06DFE00287FF4B0AE0220FFF7E2
:100B1000EDFC00283FF4AAAE049800F0CBFE05904F
:100B2000E6E70023642104A8049300F059FE00289E
:100B30007FF49CAE0220FFF7D9FC00283FF496AE6C
:100B4000049800F0B9FEEAE70220FFF7CFFC002886
:100B50003FF48CAE00F0C8FEE1E70220FFF7C6FCD0
:100B600000283FF483AE05A9142000F0C3FE074619
:100B70000421049004A800F03DFE3946B9E7322074
:100B800000F01AFE071EFFF671AEBB077FF46EAED3
:100B9000384A07EB0903926893423FF667AE02209A
:100BA000FFF7A4FC00283FF461AE27F003074F4491
:100BB000B9453FF4A5AE484609F1040900F04CFEE2
:100BC0000421059005A800F015FEF1E74FF47A70B6
:100BD000FFF78CFC00283FF449AE00F075FE0028BA
:100BE00044D00A9B01330BD008220AA9002000F050
:100BF000FFFE00283AD02022FF210AA800F0F0FED4
:100C0000FFF77CFC1C4804F003FF13B0BDE8F08F35
:100C1000002E3FF42BAE0BF00B030B2B7FF426AE14
:100C20000023642105A8059300F0DAFD074600289B
:100C30007FF41CAE0220FFF759FC804600283FF4E9
:100C400015AEFFF75BFC41F2883004F0E1FE059839
:100C500000F05CFF46463C4600F00EFFA0E506466D
:100C60004EE64FF0000901E6BA467EE637467CE6DE
:100C70008C23002000230020A0860100094A49F2AD
:100C80006900136899B21B0C00FB013344F25061F8
:100C90001360054B186882B2000C01FB020018605B
:100CA00080B270471423002010230020002110225E
:100CB00010B5044600F094FE034B03CB2060616046
:100CC0001868A06010BD00BF00E8F11F2DE9F041D9
:100CD000ADF5527D0D46002140F2751270AC07460D
:100CE00012A8119100F07CFE4FF4C472002120463E
:100CF00000F076FE0DF1440802F0A6FB4FF47A7284
:100D0000264BB0FBF2F0186093E80700022384E85A
:100D100007000DF5F1702382FFF7C8FF47F60503C2
:100D20001F4907A8238407F057F925230DF2F32262
:100D30000DF13C0C84F8323107AB1E46083203CE6D
:100D4000664542F8080C42F8041C3346F5D1306879
:100D500041461060204633791371012200F058FF9C
:100D6000002380B2E97E0393AB7E029305F1190361
:100D700001930123009307A3D3E90023CDE9048065
:100D8000384602F01FFF0DF5527DBDE8F08100BF2F
:100D9000AFF300809E6AC421818A46EE9824002029
:100DA000E87F00082DE9F0412C4CDAB080460D4672
:100DB000237A5BBB27A9284601F04EF80746002896
:100DC00042D19DF89D60C82E3ED801464FF4A662E0
:100DD000204600F005FE4FF4807332460DF19E016F
:100DE000C4F8F8314FF4007304F109002644C4F844
:100DF0000C334FF44073C4F8203400F0CBFD9DF861
:100E00009C30777223720BB9EB7E237206AC812281
:100E1000002127A800F0E4FD0122214627A801F0C7
:100E200061F8002380B2E97E0393AB7E029305F163
:100E3000190301932823CDE904400093404605A3FC
:100E4000D3E9002302F0BEFE5AB0BDE8F08100BF36
:100E5000AFF3008026417272DF25D7B7605E0020B5
:100E6000F0B5254E4FF48A75F1B0002405FB0065FE
:100E700096F8D830D822214685F8DC303AA885F893
:100E8000E84006AF00F0ACFD06F1090000F0A0FD5F
:100E9000D5F8E430C2B206F109018DF8F0000DF189
:100EA000F100CDE93A3400F075FD394601223AA847
:100EB00001F04EF8082380B2317ACDE904700127A1
:100EC0000E48CDE9023706F1D80301933023009391
:100ED00007A3D3E9002302F075FEA04206DD02F06D
:100EE000B3FAC5F8E000384671B0F0BD2046FBE724
:100EF00078F6339F93CACD8D605E0020B034002019
:100F00002DE9F04F264F87B0DFF8A080254E3846F8
:100F100002F084FE034600283AD00024224DADF8AA
:100F20001440A1460294A246CDE90344027B8DF809
:100F3000142003AA9968406803C21B6843F0004369
:100F400002932B6804F5A664D3F810B002F07EFA81
:100F500010EB0802CDF800A0284605F5A65541F192
:100F6000000302A9D8470028C8BF49F00109B4F519
:100F7000266FE6D1B9F1000F05D0384602F052FED7
:100F800086F800A0C3E73378072B04D80133337009
:100F900007B0BDE8F08F024802F044FEF8E700BF5A
:100FA000B034002095630020E034002040420F0060
:100FB00070B50D4614461E4602F060FD50B9022E73
:100FC00010D1012C0ED112A3D3E900230120C5E9D1
:100FD000002307E0282C10D005D8012C09D0052CBF
:100FE0000FD0002070BD302CFBD10BA3D3E9002320
:100FF000ECE70BA3D3E90023E8E70BA3D3E9002335
:10100000E4E70BA3D3E90023E0E700BFAFF30080E0
:10101000401DA12026812A0B78F6339F93CACD8DDF
:101020009E6AC421818A46EE26417272DF25D7B7B7
:10103000F017304A39059E5638B505460E4C00214A
:10104000013500F02FFCA4F82C55B4F82C0500F065
:1010500011FC78B1B4F82C0500F01CFC014648B92D
:10106000B4F82C0500F01EFCB4F82C350133A4F8BC
:101070002C35EAE738BD00BF605E0020F8B50D4CA6
:1010800002260D4FA4F5805343F8307C237E3BB9F4
:1010900065692DB1284601F065F8284601F09EF9F2
:1010A0002046A4F5A65401F05DF8012E00D1F8BD4C
:1010B0000126E7E7D0590020B08000082DE9F04F65
:1010C0008FB005460C4600AF02F0D8FC002849D18D
:1010D000237E022B1BD1E38A012B18D102F0B4F935
:1010E0000646FFF7CBFD03464FF4C87006F51676AB
:1010F000DFF8C082B3FBF0F202FB103316FA83F381
:10110000C8F80030E37E33B9A34B00221A703C3795
:10111000BD46BDE8F08F07F12401204600F050FEE7
:101120000028F4D107F11400FFF7C0FD97F826401E
:1011300007F1140107F12700224606F01BFF0028E3
:10114000E2D10F2C08D8944B1C70D8F80030A3F5CE
:101150001673C8F80030DAE797F82410284602F032
:1011600085FCD4E7E38A282B2BD010D8012B23D081
:10117000052BCCD1BFF34F8F8849894BCA6802F445
:10118000E0621343CB60BFF34F8F00BFFDE7302B0E
:10119000BDD1844EE17E327A9142B8D1607E314633
:1011A000002291F8DC50854200F0A580013201F563
:1011B0008A71042AF5D1AAE721462846FFF786FD61
:1011C000A5E721462846FFF7EDFDA0E7B2F8EC5071
:1011D0007B6005F103094FEA99094FEA8902D11DA5
:1011E000C908A8EBC10300219D46EB46584600F014
:1011F000F7FB04F1EE012A465846314400F0CAFBE1
:101200007B6813B9012000F025FB96F8D20000F0AE
:1012100031FB044630B9307200F056FB204600F036
:1012200019FBB1E0D6F8D4203AB996F8D200B6F856
:101230002C25824201D8FFF7FFFED6F8D4202A449D
:10124000944208D296F8D200B6F82C25013082429A
:1012500001D8FFF7F1FE5FFA89F25946706800F095
:10126000C7FB08B9C54679E0726896F8D2002A44EF
:101270007260D6F8D42005EB0209C6F8D49000F0CD
:10128000F9FA814509D396F8D220D6F8D400013274
:10129000001B86F8D220C6F8D400FF2D0FD80024FA
:1012A000347200F011FB204600F0D4FA00F0E0FEAA
:1012B0003D4B188108B9FFF77FF9C54627E7BB68A2
:1012C00096F8D9000AFB0362FB68D2F8E41082F8B2
:1012D000E83001F58061C2F8E030C2F8E410FFF7B1
:1012E000BFFDFFF70DFE96F8D920013202F0030290
:1012F00086F8D920B6E74FF48A7A20460AFB02F531
:1013000005F1EA01314400F057FEF86000287FF44F
:10131000FEAE0122354485F8E82002F095F8D5F8B4
:10132000E020D6ED007A801A40F6B832B8EE677A3F
:10133000DFED1E6A192838BF1920904228BF1046D9
:1013400007EE900AF8EEE77A67EEA67ADFED186A04
:10135000E7EE267AFCEEE77AC6ED007A96F8D93009
:10136000BB60BA6873680AFB02F4321992F8E8109D
:1013700059B1D2F8E410E8468B423FF427AF002180
:1013800082F8E810C2F8E010C5467368064A9B0A66
:1013900001331381BBE600BFA934002000ED00E05B
:1013A0000400FA05605E002098240020CDCCCC3DDE
:1013B0006666663FAC340020014B1870704700BF72
:1013C000A424002038B54FF00054144B22689A42F0
:1013D00022D1607DF8B1124B0025C9221149187045
:1013E0001148237D0930C0F8DB5000F8013C4FF470
:1013F0008073C0F8EF314FF40073C0F803334FF43B
:101400004073C0F8173400F0C5FAE02229462046A0
:1014100000F0E6FA012038BD0020FCE79AAD44C593
:10142000A424002016000020605E002037B500F0E4
:101430001FFE1F4C1F4D022301221F496B712368A1
:10144000288120465B68984704F5805301221A4999
:10145000D3F8C03404F5A6505B68984700231749B9
:101460004FF480520193164B16480093164B02F02E
:10147000D5FA164B197811B1124802F0F7FA01F0BB
:10148000E3FF0446FFF7FAFB4FF4C873B0FBF3F237
:1014900002FB130304F5167010FA83F00C4B18606E
:1014A00005F082F808B10F232B8103B030BD00BFD7
:1014B000E03400209824002040420F00A82400209F
:1014C000B10F0008B0340020BD100008A424002093
:1014D000AC3400202DE9F04F00242DED028B93B0A9
:1014E0000DF12C084FF0010ADFF814B2FFF708FDE8
:1014F0000A94ADF834400B94C8F804409FED798B02
:1015000000267E4D37462B680DF11D0207A928469F
:101510008DF81CA08DF81D408DED008BD3F8089040
:101520000023C8479DF81C90B9F1000F1ED010226F
:1015300000210EA800F054FA2B6808AA0AA95F69D6
:1015400028460DF11E03B8470FAB4F4698E803003D
:1015500083E803009DF834300EA958468DF84430D6
:101560000A9B0E93DDE9082302F03AFD06F5A66614
:1015700005F5A655B6F5266FC5D1002FC0D1604838
:1015800002F07CFA00283FD15E4E01F05DFF336827
:10159000984239D301F058FF0546FFF76FFB4FF42F
:1015A000C8738DF82870B0FBF3F202FB130305F546
:1015B000167010FA83F03060534E377817B9012354
:1015C0008DF82830C7F110050EA8FFF76FFB0EABA2
:1015D000EDB20DF12900D919062D28BF06252A469E
:1015E000013500F0D7F90AABEDB245480393182353
:1015F00004950293454B0193012300933BA3D3E948
:10160000002302F081FA347001F01EFF404A414D80
:101610001368C31AB3F57A7F2FD3106001F016FF59
:1016200002460B46364802F007FB354802F026FA20
:1016300018B32B7A0EAF384E002B14BF03230223AE
:10164000737101F001FF4FF47A7301223946B0FB48
:10165000F3F03060304600F08BFB182380B2029329
:101660002E4B019340F25513CDE9037000932448AB
:1016700020A3D3E9002302F047FA2B7A93B101F0BB
:10168000E3FE002607464FF48A7895F8D9003044E7
:1016900000F0030008FB005393F8E82072B1013614
:1016A000042EF2D1C82004F0B3F92B7A002B7FF47A
:1016B00017AF13B0BDEC028BBDE8F08FD3F8E0207C
:1016C00042B12B68BA1AFA2B38BFFA230533B2EBB2
:1016D000430FE4D3FFF7C4FB0028E0D1E2E700BFEB
:1016E000AFF300800000000000000000401DA120BA
:1016F00026812A0BF1C6A7C1D068080FE03400206C
:10170000B0340020AC340020A9340020A8340020DC
:1017100090630020605E00209824002094630020E5
:1017200010B5074C204601F053F904F5A65001F01E
:101730004FF9044A04490020BDE8104006F006BCF9
:10174000E0340020F06300207D1000082DE9F84F00
:101750004FF47A7306460D46002402FB03F7DFF8C8
:101760005080DFF8509098F900305FFA84FA5A1CE4
:1017700001D0A34212D159F824002A463146036809
:10178000D3F820B03B46D847854207D1074B01200C
:1017900083F800A0BDE8F88F0124E4E7002CFBD01B
:1017A0004FF4FA7004F034F90020F3E7DC63002012
:1017B000182300201C230020002307B50246012126
:1017C0000DF107008DF80730FFF7C0FF20B19DF83D
:1017D000070003B05DF804FB4FF0FF30F9E70000AD
:1017E0000A46042108B5FFF7B1FF80F00100C0B23E
:1017F000404208BD074B0A4630B41978064B53F8EF
:101800002140014623682046DD69044BAC4630BCCC
:10181000604700BFDC6300201C230020A08601007D
:1018200070B50A4E00240A4D04F020FC3080286870
:101830003388834208D904F015FC2B680444013333
:10184000B4F5003F2B60F2D370BD00BFDE63002013
:101850009863002004F0D8BC00F1006000F500306F
:101860000068704700F10060920000F5003004F05D
:1018700059BC0000054B1A68054B1B889B1A834214
:1018800002D9104404F0EEBB00207047986300209A
:10189000DE630020024B1B68184404F0E9BB00BF64
:1018A00098630020024B1B68184404F0F3BB00BF90
:1018B000986300200020704700F1FF5000F58F1062
:1018C000D0F8000870470000064991F8243033B181
:1018D00000230822086A81F82430FFF7C3BF0120E3
:1018E000704700BF9C630020014B1868704700BF21
:1018F0000010005C194B01380322084470B51D68C4
:10190000174BC5F30B042D0C1E88A6420BD15C6847
:101910000A46013C824213460FD214F9016F4EB1C0
:1019200002F8016BF6E7013A03F10803ECD18142BA
:101930000B4602D22C2203F8012B0424094A1688F4
:10194000AE4204D1984284BF967803F8016B013C03
:1019500002F10402F3D1581A70BD00BF0010005C00
:10196000242300203C8000087047000070470000DE
:101970007047000070B504464FF47A764CB1412CA4
:10198000254628BF412506FB05F0641B04F040F8FE
:10199000F4E770BD002310B5934203D0CC5CC4546F
:1019A0000133F9E710BD0000013810B510F9013F0F
:1019B0003BB191F900409C4203D11AB10131013A87
:1019C000F4E71AB191F90020981A10BD1046FCE70F
:1019D00003460246D01A12F9011B0029FAD17047BA
:1019E00002440346934202D003F8011BFAE7704712
:1019F0002DE9F8431F4D14460746884695F82420E4
:101A000052BBDFF870909CB395F824302BB920229C
:101A1000FF2148462F62FFF7E3FF95F82400414677
:101A2000C0F1080205EB8000A24228BF2246D6B2D0
:101A30009200FFF7AFFF95F82430A41B17441E4413
:101A40009044E4B2F6B2082E85F82460DBD1FFF7AB
:101A50003BFF0028D7D108E02B6A03EB82038342C7
:101A6000CFD0FFF731FF0028CBD10020BDE8F883AD
:101A70000120FBE79C630020024B1A78024B1A708E
:101A8000704700BFDC6300201823002038B51A4CD3
:101A90001A4D204603F0DCFA2946204603F004FBE9
:101AA0002D684FF47A70D5F89020D2F8043843F0BE
:101AB0000203C2F80438FFF75DFF1149284603F01E
:101AC00001FCD5F890200F4DD2F80438286823F097
:101AD00002030D49A042C2F804384FF4E1330B6011
:101AE00001D003F013FA6868A04204D00649BDE8AB
:101AF000384003F00BBA38BD586B0020FC82000858
:101B0000048300081C230020C46300200C4B70B524
:101B10000C4D04461E780C4B55F826209A420DD0E9
:101B20000A4B002118221846FFF75AFF04600146AD
:101B300055F82600BDE8704003F0E8B970BD00BF5D
:101B4000DC6300201C230020586B0020C4630020AD
:101B5000F8B571B6002301201A46194602F0AEFE10
:101B60000446802004F0EEFB002849D00025254AD9
:101B700080274FF4D06C3D26136913F0C06F26D137
:101B8000D2F8103113F0C06F21D1236805F1006144
:101B900099602368D86023685F602368C3F800C039
:101BA00021680B6843F001030B6021680B6823F088
:101BB0001E030B6021680B68DB07FCD4237B803598
:101BC000616806FA03F3B5F5001F0B60D4D1204617
:101BD00002F0B4FEB5F5001F11D000240A4E0B4DE3
:101BE000012004F011FB3388A34205D92868204462
:101BF000013404F04FFAF6E7002004F005FB61B66B
:101C0000F8BD00BF00200052DE6300209863002072
:101C10002DE9F3470D46044600219046284640F240
:101C20007912FFF7DDFE234620220021284604F129
:101C3000220702F077F9231D022220212846C02620
:101C400002F070F9631D03222221284602F06AF98E
:101C5000A31D03222521284602F064F904F108039C
:101C600010222821284602F05DF904F11003082211
:101C70003821284602F056F904F1110308224021C8
:101C8000284602F04FF904F11203082248212846A1
:101C900002F048F904F1140320225021284602F0F2
:101CA00041F904F1180340227021284602F03AF964
:101CB00004F120030822B021284602F033F904F190
:101CC00021030822B821284602F02CF931460836B3
:101CD0003B4608222846013702F024F9B6F5A07FDA
:101CE000F4D194F83230314604F1330A00268DF8ED
:101CF000073008220DF10703284602F013F99DF87A
:101D000007304FEAC6099E4209F5A47720D394F81C
:101D10003231502B28BF50238DF80730B8F1000F17
:101D200008D1394609F24F170DF10703072228465B
:101D300002F0F8F8002604F233149DF8073007EBA0
:101D4000C6019E420DD30731C80802B0BDE8F08736
:101D50000AEB0603082239462846013602F0E2F86B
:101D6000CDE7A31908222846013602F0DBF8E4E7A4
:101D700013B5044608460021202223460190016045
:101D8000C0F8031002F0CEF8231D01980222202192
:101D900002F0C8F8631D01980322222102F0C2F864
:101DA000A31D01980322252102F0BCF8019804F13B
:101DB00008031022282102F0B5F8072002B010BD58
:101DC000F7B5047F05460E462CB1838A122B02D943
:101DD000012003B0F0BD00230722284600961946D3
:101DE00001F064FF731C01220721009328460023A1
:101DF00001F05CFFD4B9B31C0522082128460093EA
:101E000023460D2401F052FFB378102BE0D837465B
:101E1000BB1BB278934210D307342B7FA88AE40807
:101E2000B3B9844294BF00200120D2E7AB8A0824D2
:101E3000DB00083BDB08B370E6E7FB1C2146082209
:101E40002846009300230834013701F02FFFDFE715
:101E5000201A18BF0120BCE7F7B5047F05460E46DF
:101E60002CB1838ACA2B02D9012003B0F0BD002314
:101E7000082228460096194601F018FF731CD4B9B1
:101E800008220093234610241146284601F00EFF35
:101E90007378C82BE8D801235F1C7278013B93420A
:101EA00010D307342B7FA88AE408B3B9844294BFC7
:101EB00000200120D9E7AB8A0824DB00083BDB08BF
:101EC0007370E5E7F31921460822284600930023A2
:101ED00001F0ECFE08343B46DEE7201A18BF012073
:101EE000C3E70000F7B50D46044600211646284614
:101EF0008122FFF775FD234608220021284602F0C3
:101F000011F894F901206378002AB8BF7F238DF877
:101F100007309EB90F270DF1070307220821284635
:101F200002F000F8002602349DF8073007EBC601E6
:101F30009E4205D30731C80803B0F0BD0827F1E77A
:101F4000A31908222846013601F0ECFFECE7000057
:101F5000F7B50E460546002114463046CE22FFF75F
:101F60003FFD2B4628220021304601F0DBFF2B7A73
:101F7000C82B28BFC8238DF807308CB930240DF149
:101F8000070308222821304601F0CCFF2F467B1B97
:101F90009DF80720934205D3E01DC00803B0F0BDB3
:101FA0002824F3E707F109032146082230460834C4
:101FB000013701F0B7FFEAE7F7B5047F05460E46A3
:101FC00034B1838AB3F5827F02D9012003B0F0BD1A
:101FD0000123102200212846009601F067FEDCB99B
:101FE000B31C09221021284600932346192401F02E
:101FF0005DFE7388B3F5807FE7D83746BB1B7288D8
:10200000934210D307342B7FA88AE408B3B98442E3
:1020100094BF00200120D9E7AB8A1024DB00103BDD
:10202000DB087380E5E73B1D214608222846009324
:1020300000230834013701F039FEDFE7201A18BF0A
:102040000120C3E730B50A44084D91420DD011F884
:10205000013B5840082340F30004013B2C4013F09F
:10206000FF0384EA5000F6D1EFE730BD2083B8EDDE
:10207000F7B5364A6B46106851686A4603C30823B1
:102080003349344805F086FF044690BB0A25324A9E
:102090006B46106851686A4603C308232F492D48D0
:1020A00005F078FF0446002847D00369B3F5F01F18
:1020B00043D8B0F86620B2F5AF6F3ED1284A02444B
:1020C00002F15C018B4238D35C3B224900209E1A0E
:1020D000FFF7B8FF04F16401074632460020FFF71E
:1020E000B1FFA3689F4228D1E368984208BF00254A
:1020F00023E00369B3F5F01F26D8428BB2F5AF6F2A
:1021000020D1174A024402F110018B4218D3103B30
:10211000104900209D1AFFF795FF04F118010646AB
:102120002A460020FFF78EFFA3689E4202D1E36893
:10213000984201D00D25AAE70025284603B0F0BD3E
:102140001025A4E70C25A2E70B25A0E74C8000088A
:10215000DCFF1D00000002085580000890FF1D00F4
:102160000800FEF710B5037C044613B9006804F0BC
:102170001DF9204610BD00000023BFF35B8FC36034
:10218000BFF35B8FBFF35B8F8360BFF35B8F7047E1
:10219000BFF35B8F0068BFF35B8F704770B5054678
:1021A0000C30FFF7F5FF044605F108063046FFF74F
:1021B000EFFFA04206D96D683046FFF7E9FF2544DE
:1021C000281A70BD3046FFF7E3FF201AF9E7000038
:1021D00070B505464068A0B105F10C0605F1080090
:1021E000FFF7D6FF04463046FFF7D2FF844204F1E2
:1021F000FF34304694BF6D680025FFF7C9FF2C44BB
:10220000201A70BD38B50C460546FFF7C7FFA0423F
:1022100010D305F10800FFF7BBFF04446868BFF363
:102220005B8FB4FBF0F100FB11440120AC60BFF305
:102230005B8F38BD0020FCE72DE9F04114460746CE
:102240000D46FFF7C5FF844228BF0446D4B1B84607
:1022500058F80C6B4046FFF79BFF3044286040461F
:102260007E68FFF795FF331A9C4203D801206C600B
:10227000BDE8F081A41B6B603B682044AB60E86064
:102280000220F5E72046F3E738B50C460546FFF790
:102290009FFFA04210D305F10C00FFF779FF044423
:1022A0006868BFF35B8FB4FBF0F100FB11440120C1
:1022B000EC60BFF35B8F38BD0020FCE72DE9FF41E8
:1022C0008846694607466C46FFF7B6FF002506B20A
:1022D00004EBC606B4420AD0626808EB0501206828
:1022E0000834FFF757FB54F8043C1D44F2E7294635
:1022F0003846FFF7C9FF284604B0BDE8F08100006A
:10230000F8B505460C300F46FFF742FF05F1080609
:1023100004463046FFF73CFFA042304688BF6C6859
:10232000FFF736FF201A386020B12C683046FFF7DF
:102330002FFF2044F8BD000073B5144606460D4635
:10234000FFF72CFF8442019028BF0446DCB101A9AD
:102350003046FFF7D5FF019B33B93268C5E9023338
:10236000C5E9002401200CE09C42286038BF01949C
:10237000019884426860F5D93368241A0220AB6062
:10238000EC6002B070BD2046FBE700002DE9FF4184
:102390000F4669466C46FFF7CFFF00B2002604EBFC
:1023A000C005AC4209D0D4F80480B81954F8081B11
:1023B00042464644FFF7EEFAF3E7304604B0BDE884
:1023C000F081000038B50546FFF7E0FF04460146FE
:1023D0002846FFF717FF204638BD000008B103F07C
:1023E000E5BF70477047000010B4134602681468D8
:1023F0000022A4465DF8044B6047000000F58050C1
:1024000090F859047047000000F5805090F852048D
:102410007047000000F5805090F9580470470000A4
:102420004E207047302383F3118800F58052D2F894
:102430009C34D2F898041844D2F894341844D2F852
:102440007C341844D2F88C341844D2F888341844B8
:10245000002383F31188704700F58050C0F85414AE
:10246000012070472DE9F04F0C4600F5805185B0F2
:102470001F4691F8523405469046BDF838909BB1FE
:10248000D1F878340133C1F878342368980006D441
:10249000237B082B0BD9627B0AB10F2B07D9D1F80C
:1024A0007C340133C1F87C344FF0FF3010E030232E
:1024B00083F31188EB6AD3F8C42012F4001B0AD00E
:1024C000D1F8803400200133C1F8803480F31188C2
:1024D00005B0BDE8F08F20684822D3F8C43000284A
:1024E000C3F3044A6B6AB4BF40F08040800412FB1F
:1024F0000A334FEA4A161860226852004FEA0A620D
:1025000044BF40F000501860207B42EA00425A600D
:10251000607B10B342F440125A60D1F8B02401320B
:10252000C1F8B024AA1902F58352117B41F02001B1
:102530001173207B039300F0E3FF0330039B8010B3
:102540005FFA8BF20BF1010B82420DDA04EB820190
:1025500003EB820249689160F2E7AA1902F58352FF
:10256000117B60F34511E3E70122EB6A05EB4A11A9
:1025700002FA0AF201F58251C3F8D020AB191831E2
:1025800004F10C0203F58253C3E90487234653F890
:10259000040B934241F8040BF9D11B882E440B80A5
:1025A00041F2680346F803A006F5805609F00303DC
:1025B00096F86C2043F0100322F01F02134386F8B4
:1025C0006C30002383F3118842463B46214628465F
:1025D000CDF8009000F05AFF012079E72DE9F0478F
:1025E00000F58056044696F85254002D40F00381C1
:1025F000037C032B40F0948028462B462F465FFA3D
:1026000080FC944510DA01EBCC0E51F83CC0BCF1D3
:10261000000F04DBDEF804C0BCF1000F02DB013761
:102620000130ECE70133FBE7302080F31188E06AEA
:10263000F3B9D0F8803043F00203C0F880304E2365
:10264000E06A002F6FD1D0F8803043F00103C0F86A
:1026500080306A4B6A4A1B6803F1805303F52C53A0
:102660009B009342A36240F2B080664800F0E6FE11
:102670004D2B42D8DFF884814FEA034EDFF8889172
:10268000D8F800C04EEA8C0EC0F884E00CF18050FF
:1026900000F52C508000606103EB0C00D4F82CC0D6
:1026A000C3F14E03C8F80000DCF8800040F03000B1
:1026B000CCF880004FF0000CD4F81480E6465FFAA6
:1026C0008CF08242BCDD01EBC00A51F830000028DA
:1026D00010DBDAF804A0BAF1000F0BDA09EA0040C7
:1026E0000AF07F0A40EA0A0040F0084048F82E004D
:1026F0000EF1010E0CF1010CE1E7836923F00103F7
:10270000836100F0A1FE0646E36A9B69D90704D500
:1027100000F09AFE831BFA2BF6D9002383F311886D
:102720002846BDE8F087B7EB530F3DD2DFF8CCE089
:102730004FEA074CDEF800304CEA830CC0F888C042
:1027400003F1805003EB4703002700F52C50CEF82F
:102750000030BC468000A061E06AD0F8803043F0D1
:102760000C03C0F88030D4F818E0FBB29A427FF72F
:1027700070AF51F8330001EBC3080028D8F80430DB
:1027800001DB002B0EDB20F0604023F0604340F0C3
:10279000005043F000434EF83C000EEBCC000CF12F
:1027A000010C43600137E0E7836923F00103836193
:1027B00000F04AFE0646E36A9B69DA07ADD500F0F1
:1027C00043FE831BFA2BF6D9A7E7E26A936923F04D
:1027D0000103936100F038FE0746E36A9B69DB075B
:1027E00005D500F031FEC31BFA2BF6D995E701257C
:1027F00086F8525491E7002592E700BFEC63002071
:10280000FCB50040608000080000FF0713B500F52C
:1028100080540191606CFFF7DBFC1F280AD920224D
:102820000199606CFFF74AFDA0F12003584258411E
:1028300002B010BD0020FBE708B5302383F31188F8
:1028400000F58050406CFFF797FC002383F311885C
:1028500008BD0000002202608281426082607047F1
:102860000022002310B5C0E90023002304460C30E9
:1028700020F8043CFFF7EEFF204610BD2DE9F0479D
:102880009A4688B0074688469146302383F31188DC
:1028900007F580546846FFF7E3FF606CFFF77EFCA6
:1028A0001F282ED920226946606CFFF78BFD202857
:1028B00027D194F8523423B303AD444605AB2E46DA
:1028C000083403CE9E4244F8080C44F8041C3546F4
:1028D000F5D130682060B388A380DDE90023C9E921
:1028E0000023BDF80830AAF80030002383F31188D4
:1028F00053464A464146384608B0BDE8F04700F026
:10290000B3BD002080F3118808B0BDE8F087000057
:102910002DE9F84F0023064600F581540546884608
:102920001034C0E90133274B46F8303B3746384670
:102930002037FFF795FFA742F9D105F580544FF4F2
:10294000805305F5A3594FF0000A266300266764FB
:1029500005F5835709F110094FF0000B1037E663B6
:10296000C4E90D36012384F8403084F84830A7F1DB
:102970001800203747E910ABFFF76CFF47F8286CC9
:102980004F45F4D1B8F1010F84F85884A4F85A6483
:10299000A4F85C64A4F85E6484F86064A4F86264DB
:1029A000A4F86464A4F8666484F8686402D90648EC
:1029B00000F044FD054B284653F82830EB62BDE893
:1029C000F88F00BFB080000884800008A080000855
:1029D000044B10B5197804464A1C1A70FFF798FF8B
:1029E000204610BDE96300202DE9F04300295AD0AC
:1029F0002E4E2F48B6FBF1F481428CBF0A201120E5
:102A0000431EB4FBF0F700FB1740DDB220B1022BF0
:102A10001846F5D8002032E07B1EB3F5806F2ED229
:102A2000C5EBC5084FF47A7308F103044FEAE40ECE
:102A3000C4F3C7040EF10109281B0EFB033E5FFA25
:102A400080FC59FA80F0BEFBF0F0B0F5617F18DC35
:102A500083B2601C5CFA80F07843B6FBF0F08142F0
:102A6000D8D1611E0F29D5D80CF1FF310729D1D853
:102A70000120138057801071547182F806C0BDE8A0
:102A8000F08308F1FF34E010C4F3C70400F1010E35
:102A90002D1B00FB03335FFA85FC5EFA85F5B3FB63
:102AA000F5F39BB2D5E70846E9E700BF00B4C404DC
:102AB0003F420F0030B50D4B05200D4D1C786C4387
:102AC0008C420ED159780120518099785171D97872
:102AD0009171197911715B7903EB83035B001380AA
:102AE00030BD013803F10603E8D1F9E7F0800008B2
:102AF00040420F0038B540F27772C36A154CC3F8F4
:102B0000BC200722C36AC3F8C8202268C16A9300A8
:102B100043F4C023C1F8A03002F1805302F16C01EC
:102B2000C56A03F52C53EA3289009B00226041F00C
:102B3000E061094AC361C5F8C01003F5D87103F517
:102B40006A7341629342836202D9044800F076FCC2
:102B500038BD00BFEC630020FCB500406080000879
:102B60002DE9F04F00F580551F4689B0044695F8D1
:102B7000583489469046022B04D90026304609B0C5
:102B8000BDE8F08FA84A52F8231009B942F8230093
:102B9000A648C4F80C9001782774C9B9302383F390
:102BA0001188A34BD3F8EC2042F48072C3F8EC20D8
:102BB000D3F8942042F48072C3F89420D3F8942080
:102BC00022F48072C3F894200123037081F31188EA
:102BD00095F851347BB9302383F31188954A95F8E1
:102BE0005834D35C0BB3012B28D0012385F8513422
:102BF000002383F31188302383F31188E26A9369F9
:102C000023F01003936100F01FFC8246E36A9E6983
:102C100016F0080619D000F017FCA0EB0A03FA2BF7
:102C2000F4D9002686F31188A8E70321132001F0C8
:102C3000A1FF0321152001F09DFFD6E703211420F9
:102C400001F098FF03211620F5E79A6942F001028E
:102C50009A6100F0F9FB8246E36A9A69D00706D4CC
:102C600000F0F2FBA0EB0A03FA2BF5D9D9E79A6939
:102C70004FF0000A42F002029A61E36AC3F854A0DE
:102C80008AF3118804F5825B686CFFF775FA0BF123
:102C9000100B202200216846FEF7A2FE02A8FFF7D3
:102CA000D9FD6A460BEB06030DF1180ECDF818A0FE
:102CB00094460833BCE80300F44543F8080C43F895
:102CC000041C6246F4D1DCF8000020361860B6F52A
:102CD000806F9CF804201A71DBD1002304F5A25206
:102CE000494620461A3285F8503485F85334FFF7A8
:102CF0007BFE064690B9E26A936923F00103936173
:102D000000F0A2FB0546E36A9B69D9077FF535AF62
:102D100000F09AFB431BFA2BF5D92EE795F85E34A9
:102D2000C5F86C94591E95F85F34E26A013B1B02AA
:102D300043EA416395F8601401390B43B5F85C141C
:102D4000013943EA0143D361B8F1000F36D004F5ED
:102D5000A352414620460232FFF7ACFE90B9E26A28
:102D6000936923F00103936100F06EFB0546E36A6B
:102D70009B69DA077FF501AF00F066FB431BFA2B76
:102D8000F5D9FAE695F86724C5F87084511E95F8D0
:102D90006824E36A013A120142EA012295F86614B6
:102DA00001390A43B5F86414013942EA014242F498
:102DB0000002DA604FF42062E36A9A64E36A4FF03B
:102DC00000082046C3F8BC80FFF794FE85F85984BC
:102DD0006FF04042E36A1A65174AE36A5A654FF09A
:102DE0000222E36A9A654FF0FF32E36AC3F8E020FB
:102DF0000322E36A9742DA653FF4C0AEE26A936960
:102E000023F00103936100F01FFB0746E36A9B690F
:102E1000DB0705D500F018FBC31BFA2BF6D9ACE68F
:102E2000012385F85234A9E6E0630020E86300201E
:102E30000044025898800008550200022DE9F04F26
:102E4000054689B090469946002741F2680A00F588
:102E50008056EB6AD3F8D830FB40D80751D505EB44
:102E600047124FEA471B52441379190749D4D6F841
:102E700084340133C6F8843405F5A553C3E90089C9
:102E800013799A0605EB0B0248BFD6F8B4345244C6
:102E900044BF0133C6F8B434137943F00803137107
:102EA000DB0723D596F8533403B305F582546846FF
:102EB000FFF7D6FC03AB18345C4404F1080C20681F
:102EC000083454F8041C1A46644503C21346F6D16C
:102ED0002068694610602846A2889A800123ADF8D0
:102EE00008302B68CDE90089DB6B9847D6F8A83409
:102EF000D6F854040133C6F8A83410B103681B692E
:102F000098470137202FA4D109B0BDE8F08F000009
:102F10002DE9F04F0F468DB0044600F097FA824637
:102F20008946002F5BD1E36AD3F8A02012F4FE0F8C
:102F300003D100200DB0BDE8F08FD3F8A42092019A
:102F400041BF04F58051D1F898240132C1F898248A
:102F5000D3F8A4205606ECD0D3F8A450E669C5F304
:102F600005254823E8464FF0000B03FB0566404665
:102F7000FFF770FC326851004ABF22F06043C2F391
:102F80008A4343F00043920048BF43F080430093DC
:102F9000736813F400131BBF012304F580528DF8EE
:102FA0000D308DF80D301EBFD2F8B8340133C2F8A1
:102FB000B834F38803F00F038DF80C309DF80C0043
:102FC00000F09EFA5FFA8BF3984225D9F2180CA90B
:102FD0000BF1010B127A0B4403F82C2CEEE7012FB6
:102FE000A7D1E36AD3F8B02012F4FE0FA1D0D3F832
:102FF000B420950141BF04F58051D1F898240132E5
:10300000C1F89824D3F8B420500692D0D3F8B45025
:10301000266AC5F30525A4E7EFB9E36AC3F8A8500B
:1030200004A807ADFFF71CFC98E80F0007C52B802C
:103030000023204604A9ADF81830236804F5805415
:10304000DB6BCDE904A9984758B1D4F8903401332B
:10305000C4F890346EE7012FE2D1E36AC3F8B850A8
:10306000DEE7D4F8943401200133C4F8943461E7E6
:103070002DE9F04105460F4600F5805401263946FA
:103080002846FFF745FF10B184F85364F7E7D4F8FA
:10309000A834D4F854040133C4F8A83420B1036828
:1030A000BDE8F0411B691847BDE8F081C36AF0B57F
:1030B0001A6C12F47F0F2BD01B6C00F5805441F278
:1030C00068054FF0010CC4F8AC340023471900EB3D
:1030D00043125E012A44117911F0020F15D04907FD
:1030E00013D4B959C66A0CFA01F1D6F8CCE011EA4A
:1030F0000E0F0AD0C6F8D410117941F004011171F5
:10310000D4F88C240132C4F88C240133202BDED176
:10311000F0BD00002B4B70B51E561B5C012B30D848
:10312000294D2A4A55F8233052F8264013B349B3A3
:10313000236D9A0510D54FF40073236500F086F9CE
:1031400050EA01020B4602D0013861F10003024649
:1031500055F82600FFF772FE236D9B012CD54FF02A
:10316000007255F82630226503F58053012283F85A
:10317000592421E001232365102323654FF4805354
:10318000236570BD236DDA0702D4236D5B0706D576
:103190000523002155F826002365FFF769FF236DFD
:1031A000D80602D4236D590606D55023012155F8BF
:1031B00026002365FFF75CFF55F82600BDE8704048
:1031C000FFF774BF9C800008E0630020A080000827
:1031D00008B5302383F31188FFF768FF002383F3DA
:1031E000118808BDC36AD3F8C00010F07C5005D028
:1031F000D3F8C40080F40010C0F3405070470000C2
:1032000008B5302383F3118800F58050406CFEF739
:10321000C5FF002383F3118843090CBF0120002060
:1032200008BD000000F5805393F8592462B1C16ACB
:103230008A6922F001028A61D3F89C240132C3F822
:103240009C24002283F85924704700002DE9F7439D
:10325000302181F3118800F58251002541F2680E7A
:103260004FF00108103100F5805C00EB4514744408
:10327000267977071CD4F6061AD58E69D0F82C90DB
:1032800008FA06F6D9F8CC703E4211D04F68019783
:103290000F689742019F9F410AD2C9F8D4602679EE
:1032A00046F004062671DCF888440134CCF88844E2
:1032B00001352031202DD8D1002383F3118803B0AC
:1032C000BDE8F083F8B51E4600230F46054613708F
:1032D0001446FFF795FF80F0010038701EB12846B4
:1032E000FFF780FF2070F8BD2DE9F04F85B09946BB
:1032F0000D468046164691F800B0DDE90EA3029314
:103300001378019300F0A2F82B7804460F4613B906
:103310003378002B41D022463B464046FFF796FFCC
:10332000FFF756FFFFF77EFF4B4632462946FFF771
:10333000C9FF2B7833B1BBF1000F03D0012005B0DA
:10334000BDE8F08F337813B1019B002BF6D108F55F
:10335000805303935445029B77EB03031DD2039BD9
:10336000D3F85404C8B10368AAEB04011B6898475A
:103370004B46324629464046FFF7A4FF2B7813B14F
:10338000BBF1000FDAD1337813B1019B002BD5D1FB
:1033900000F05CF804460F46DCE70020CFE70000B1
:1033A000002108B50846FFF7B5FEBDE8084001F06A
:1033B00071B8000008B501210020FFF7ABFEBDE8A1
:1033C000084001F067B8000008B500210120FFF7B0
:1033D000A1FEBDE8084001F05DB80000012108B57C
:1033E0000846FFF797FEBDE8084001F053B800001B
:1033F00000B59BB0EFF3098168226846FEF7CAFA70
:10340000EFF30583014B9B6BFEE700BF00ED00E08F
:1034100008B5FFF7EDFF000000B59BB0EFF30981A1
:1034200068226846FEF7B6FAEFF30583014B5B6B43
:10343000FEE700BF00ED00E0FEE700000FB408B5B6
:10344000029802F08BFAFEE702F0DEBF02F0C0BF86
:1034500013B56C46031D84E8060094E8030083E876
:103460000500012002B010BD73B58568019155B10A
:103470001B885B0707D4D0E900369B6B9847019AFD
:10348000C1B23046A847012002B070BDF0B58668D1
:1034900089B005460C465EB1BDF838305B070AD4EA
:1034A000D0E900379B6B98472246C1B23846B047F7
:1034B000012009B0F0BD0022002301F10806CDE98A
:1034C000002300230A46ADF8083003AB1068083229
:1034D00052F8041C1C46B24203C42346F6D11068BD
:1034E00020609288A280FFF7B1FF0423ADF8083076
:1034F0002B68CDE90001DB6B694628469847D7E782
:10350000082817D909280CD00A280CD00B280CD071
:103510000C280CD00D280CD00E2814BF40203020D1
:1035200070470C20704710207047142070471820F7
:1035300070472020704700002DE9F041456A15B919
:103540004162BDE8F0814B68AC4623F06047C3F3AD
:103550008A464FEAD37EC3F3807816EA230638BF43
:103560003E462B465A68BEEBD27F22F060440AD01A
:10357000002A18DAA40CB44217D19D420FD10D6075
:10358000DEE71346EEE7A74207D102F08044C2F31C
:10359000807242450BD054B1EFE708D2EDE7CCF88A
:1035A00000100B60CDE7B44201D0B442E5D81A68F0
:1035B0009C46002AE5D11960C3E700002DE9F047D9
:1035C000089D01F0070400EBD1004FF47F494FEA5A
:1035D000D508224405F00705944201D1BDE8F087E3
:1035E00004F0070705F0070A111B08EBD50E574535
:1035F0003E4613F80EC038BF5646C6F108068E4246
:1036000028BF0E46E108415C34443544B94029FAEC
:1036100006F721FA0AF1FFB28CEA010147FA0AF72C
:1036200039408CEA010C03F80EC0D5E780EA01208E
:10363000082341F2210201B2013B4000002980B27F
:10364000B8BF504013F0FF03F5D1704738B50C46B2
:103650008D18A54200D138BD14F8011BFFF7E6FF15
:10366000F7E7000042684AB11368818943604389E3
:1036700001339BB29942438138BF83811046704722
:1036800070B588B0044620220D4668460021FEF73A
:10369000A7F920460495FFF7E5FF024660B16B46A7
:1036A000054608AE1C46083503CCB44245F8080C64
:1036B00045F8041C2346F5D1104608B070BD000043
:1036C000082817D909280CD00A280CD00B280CD0B0
:1036D0000C280CD00D280CD00E2814BF4020302010
:1036E00070470C2070471020704714207047182036
:1036F0007047202070470000082817D90C280CD9E3
:1037000010280CD914280CD918280CD920280CD929
:1037100030288CBF0F200E207047092070470A20E8
:1037200070470B2070470C2070470D207047000039
:103730002DE9F843078C0446072F1ED900254FF6C4
:10374000FF73D0E90298C5F12006A5F1200029FAFF
:1037500005F1083508FA06F628FA00F0314301436E
:103760001846C9B2FFF762FF402D0346EBD13A4637
:10377000E169BDE8F843FFF769BF4FF6FF70BDE8A8
:10378000F883000010B54B6823B9CA8A63F30902B5
:10379000CA8210BD04691A681C600361C38A013BB8
:1037A000C3824A60EFE700002DE9F84F1D46CB8A3F
:1037B0000F468146C3F30901924605290B4630D0D6
:1037C0000020AAB207F11A049EB21FFA80F8042E54
:1037D0000FD8904503F1010306D30A44FB8A62F334
:1037E00009030120FB821AE01AF800600130E65458
:1037F000EAE79045F1D2A1F1050B1C237C68BBFBE5
:10380000F3F203FB12BB1FFA8BF6002C45D148469E
:10381000FFF728FF044638B978606FF00200BDE872
:10382000F88F4FF00008E6E7002606607860ADB23A
:103830004FF0000B454510D90AEB0803221D13F881
:10384000011B08F101089155B1B21FFA88F81B2934
:103850002BD0454506F10106F1D8FB8AC3F30902D6
:10386000154465F30903BCE701321C4692B2236894
:10387000002BF9D16B1F0B441C21B3FBF1F3013377
:103880009BB29A42D3D2BBF1000FD0D14846FFF78A
:10389000E9FE20B9C4F800B0BFE70122E7E7C0F8AD
:1038A00000B05E4620600446C1E74545D5D948468C
:1038B000FFF7D8FE08B92060AFE7C0F800B00026D7
:1038C00020600446B6E700002DE9F04F1C4607468D
:1038D00088462DED028B83B05B690192002B00F0CE
:1038E0009A80238C2BB1E269002A00F09480072B88
:1038F00035D807F10C00FFF7B5FE054638B96FF073
:103900000205284603B0BDEC028BBDE8F08F1422FF
:103910000021FEF765F8228CE16905F10800FEF749
:1039200039F8208C48F00041013080B2FFF7E4FE06
:10393000FFF7C6FE013880B2208401302874384673
:103940006369228C1B782A4403F01F0363F03F0352
:10395000137269602946FFF7EFFD0125D1E74FF0AB
:10396000000900F10C034FF0800A4E464D4608EE68
:10397000103A18EE100AFFF775FE83460028BED0F5
:1039800014220021FEF72CF8002E3AD1019B0222CE
:10399000ABF808300BF1080E1FFA82FC218C0CF1F9
:1039A0000100BCF1060F80B201D88E422BD3FFF785
:1039B000A3FE8E4208BF4FF0400AFFF781FE626906
:1039C0000138013512781BFA80F1013002F01F0234
:1039D0002DB242EA491289F001094AEA020A48F086
:1039E000004281F808A059468BF810003846CBF801
:1039F00004204FF0000AFFF79FFD238CB342B8D19B
:103A00007FE70022C6E7E169895D01360EF8021002
:103A1000B6B20132C0E76FF0010572E7F8B515469E
:103A20000E463022002104461F46FDF7D9FF069BB3
:103A3000B5F5001FA760636004F11000079B34BF59
:103A40006A094FF6FF72E661A362002397B29A42B9
:103A500006D800230360A782E3822383E360F8BDD6
:103A60000660013330462036F1E7000003781BB9C9
:103A70004BB2002BC8BF0170704700000078704740
:103A8000F8B50C46C969074611B9238C002B37D10C
:103A9000257E1F2D34D8387828BB228C072A2CD8B5
:103AA000268A36F003032BD14FF6FF70FFF7CEFDC9
:103AB00020F0010031024FF6FF72400441EA056137
:103AC000400C41EA4025234629463846FFF7FCFED4
:103AD000002807DD626913780133DBB21F2B88BF32
:103AE00000231370F8BD218A2D0645EA0125054300
:103AF0002046FFF71DFE0246E5E76FF00300F1E701
:103B00006FF00100EEE7000070B58AB0044616467B
:103B10000021282268461D46FDF762FFBDF83830B7
:103B200069462046ADF810300F9B05939DF8403054
:103B30008DF81830119B0793BDF84830CDE9026528
:103B4000ADF82030FFF79CFF0AB070BD2DE9F041C1
:103B5000D36905460C4616460BB9138C5BBB377E02
:103B60001F2F28D895F80080B8F1000F26D03046D6
:103B7000FFF7DEFD337821020246284641EAC331D1
:103B8000338A41EA080141EA076141EA03413346C9
:103B900041F08001FFF798FE00280ADD3378012B01
:103BA00007D1726913780133DBB21F2B88BF002362
:103BB0001370BDE8F0816FF00100FAE76FF00300C9
:103BC000F7E70000F0B58BB004460D46174600211C
:103BD000282268461E46FDF703FF9DF84C30294613
:103BE00020465A1E534253416A468DF800309DF8D4
:103BF0004030ADF81030119B05939DF848308DF89A
:103C00001830149B0793BDF85430CDE90276ADF817
:103C10002030FFF79BFF0BB0F0BD0000406A00B101
:103C200004307047436A1A68426202691A6003618D
:103C3000C38A013BC38270472DE9F041D0F8208050
:103C400014461D46184E4146002709B9BDE8F081CB
:103C5000D1E90223A21A65EB0303964277EB030333
:103C60001ED2036A8B420DD1FFF78CFD036A1B68DD
:103C7000036203690B60C38A0161013B016AC3826D
:103C80008846E2E7FFF77EFD0B68C8F8003003695D
:103C90000B60C38A0161013BC382D8F80010D4E7EE
:103CA00088460968D1E700BF80841E002DE9F04FE7
:103CB0008BB00D4614469B46DDF850908046002898
:103CC00000F01881B9F1000F00F01481531E3F2B52
:103CD00000F21081012A03D1BBF1000F40F00A81EC
:103CE0000023CDE90833B8F81430B5EBC30F4FEA21
:103CF000C30703D300200BB0BDE8F08F2B199F4200
:103D0000D8F80C3036BF7F1B2746FFB21BB9D8F856
:103D10001030002B7AD0272D4DD8C5F1280600236E
:103D20002946B742009308ABD8F808002CBFF6B27A
:103D30003E46A7EB060A354432465FFA8AFAFFF799
:103D40003DFCB8F81430282103F10053053BDB009B
:103D50000493D8F80C300393039B13B1BAF1000F0E
:103D60002CD1D8F8100040B1BAF1000F05D008AB43
:103D70005246691A0096FFF721FC38B2002FB9D0DD
:103D800066070AD00AAB624203EBD40102F00702D5
:103D900011F8083C134101F8083C082C3DD9102CBF
:103DA00040F2B580202C40F2B780BBF1000F00F04C
:103DB0009C80082335E0BA460026C2E7049BE02B2E
:103DC00028BFE02306930B44AB42059315D95A1B39
:103DD0000398691A0096924508AB00F1040034BFBD
:103DE0005246D2B20792FFF7E9FB079A1644AAEBB4
:103DF000020A1544F6B25FFA8AFA049B069A0599FC
:103E00009B1A0493039B1B680393A5E700933A4610
:103E100008AB2946D8F80800ADE7BBF1000F13D076
:103E20000123B4EBC30F6BD0082C12D89DF82030BF
:103E3000621E23FA02F2D50706D54FF0FF3202FACE
:103E400004F423438DF820309DF8203089F80030A9
:103E500051E7102C12D8BDF82030621E23FA02F26E
:103E6000D10706D54FF0FF3202FA04F42343ADF830
:103E70002030BDF82030A9F800303CE7202C0FD8C6
:103E80000899631E21FA03F3DA0705D54FF0FF32D4
:103E900002FA04F40C430894089BC9F800302AE79E
:103EA000402C2AD0611EC4F12102A4F12103DDE9D6
:103EB000086526FA01F105FA02F225FA03F3114327
:103EC0001943CB0711D50122A4F12003C4F120012D
:103ED00002FA03F322FA01F1A2400B43524263EBD0
:103EE000430332432B43CDE90823DDE90823C9E925
:103EF000002300E76FF00100FDE66FF00800FAE62E
:103F0000082CA1D9102CB4D9202CEED8C4E7BBF1D1
:103F1000000FAED0022384E7BBF1000FBCD0042316
:103F20007FE70000012A30B5144638BF012485B070
:103F30000025402C28BF4024012ACDE9025518D87D
:103F40001B788DF8083063070AD004AB624203EB9C
:103F5000D40502F0070215F8083C934005F8083C28
:103F6000034600912246002102A8FFF727FB05B077
:103F700030BD082AE4D9102A03D81B88ADF80830D0
:103F8000E1E7202A95BF1B68D3E900230293CDE91E
:103F90000223D8E710B5CB681BB98B600B618B820D
:103FA00010BD04691A681C600361C38A013BC382A7
:103FB000CA60F0E703064CBFC0F3C0300220704770
:103FC00008B50246FFF7F6FF022806D15306C2F3F2
:103FD0000F2001D100F0030008BDC2F30740FBE74A
:103FE0002DE9F04F93B004460D46CDE903230A684E
:103FF0001046FFF7DFFF0228824614BFC2F30626F1
:104000000026002A80F2F88112F0C04940F0F481C5
:10401000097B002900F0F081022803D02378B34205
:1040200040F0ED81C2F3046310462944069302F088
:104030007F030593FFF7C4FF059B002283464FEAE9
:104040008348002348EA0A4848EA4668CE78CDE922
:104050000823F30948EA0008029368D0059B02464A
:1040600008A92046009353466768B847002800F027
:10407000C981276A4FB9414604F10C00FFF700FBE4
:10408000074690B96FF0020055E03B6998450DD0A6
:104090003F68002FF9D1414604F10C00FFF7F0FA18
:1040A00007460028EED0236A3B60276297F817C0C6
:1040B00006F01F08CCF3840CACEB0800A8EB0C0353
:1040C0001FFA80FE0028B8BF0EF120001FFA83FE01
:1040D000B8BF00B2002B0793B8BF0EF12003D7E999
:1040E0000221BCBF1BB2079352EA010338D0039BE5
:1040F0004FF0000CDFF81CE39A1A049B63EB0101FC
:1041000096457CEB01032BD36B7B97F81AE0734544
:1041100019D1029B002B78D0012821DC7868F8B9EE
:10412000DFF8ECC2944570EB010316D337E0276A41
:1041300027B96FF00C0013B0BDE8F08F3B699845CC
:10414000B4D03F68F4E7B24890427CEB010301D35E
:104150000020F0E7029B002BFAD0079B0F2B17DC07
:10416000FA7DB3003946204602F0030203F07C03D7
:104170001343FB75FFF706FB6B7BBB76029B3BB9DA
:10418000FB7DC3F38402013262F38603FB75D0E743
:104190006A7BBB7E9A42DBD1029B002B35D0B309F0
:1041A000022B32D0039B142200210DA8BB60049B7C
:1041B000FB60FDF715FC039B0AA920460A93049BAC
:1041C000ADF83EB00B932B1D8DF840A00C932B7BCC
:1041D0008DF84180013BDBB2ADF83C30069B8DF899
:1041E0004230059B8DF8433094F82C3083F0010366
:1041F0008DF84430A3689847FB7DC3F384030133F3
:1042000003F01F039B02FB82A2E7FB7DC6F3401273
:10421000B2EBD31F40F0F980C3F38403434540F071
:10422000FB80029AB6092B7B002A52D016F00106B9
:1042300061D1032B40F2F380039B394604F10C005B
:10424000BB60049BFB60FB8A66F30903AE1DFB8227
:1042500032462B7B033BDBB2FFF7A6FA00280CDAD1
:1042600039462046FFF78EFAFB7DC3F38403013302
:1042700003F01F039B02FB8204E7AB88DDE908849F
:104280003B834FF6FF73C9F12000A9F1200228FA01
:1042900009F109F1080904FA00F024FA02F20143D5
:1042A00018461143C9B2FFF7C1F9B9F1400F0346EF
:1042B000E9D1B88231462A7B033AD2B2FFF7C6F978
:1042C000FB7DB882DA43C2F3C01262F3C713FB75F9
:1042D0003EE786B92E1D013B394604F10C00DBB2E6
:1042E0003246FFF761FA0028BADB2A7B3146B88AEA
:1042F000013AD2B2E2E7F98A013BC1F30901DAB22D
:1043000004295BD8281D002307F11B069A4208D90F
:1043100010F801CB013306F801C00131DBB20529E9
:10432000F4D1039993420A9138BF043304992CBF06
:10433000002355FA83F30B9107F11B010C91796867
:104340000E930D91291DFB8AADF83EB0C3F309030E
:104350008DF840A08DF841801A44069B8DF84230BC
:10436000059BADF83C208DF8433094F82C3083F059
:1043700001038DF844300023B88A7B602A7B013A20
:10438000FFF764F93B8BB882834203D1A3680AA983
:104390002046984720460AA9FFF7FCFDFB7DBA8A14
:1043A000C3F38403013303F01F039B02FB823B8BA7
:1043B0009A420CBF00206FF01000BCE67B68002B17
:1043C000AFD0052001E01C3033461E68002EFAD124
:1043D000091A2E1D081D184401EB090C5FFA89F318
:1043E000BCF11B0F9DD89A429BD916F8013B09F1ED
:1043F000010900F8013BEFE76FF009009BE66FF061
:104400000A0098E66FF00B0095E66FF00D0092E65B
:1044100040420F0080841E006FF00E008BE66FF0AC
:104420000F0088E6EFF30983054968334A6B22F0F1
:1044300001024A6383F30988002383F311887047DC
:1044400000EF00E0302080F3118862B60D4B0E4A79
:10445000D96821F4E0610904090C0A430B49DA60C8
:10446000D3F8FC2042F08072C3F8FC20084AC2F85E
:10447000B01F116841F0010111602022DA7783F842
:104480002200704700ED00E00003FA0555CEACC5F0
:10449000001000E0302310B583F311880E4B5B68E9
:1044A00013F4006314D0F1EE103AEFF309844FF0E7
:1044B0008073683CE361094BDB6B236684F30988F6
:1044C00001F012FA10B1064BA36110BD054BFBE7DA
:1044D00083F31188F9E700BF00ED00E000EF00E092
:1044E0003F0400084204000808B5074B074A196852
:1044F00001F03D01996053680BB190689847BDE8A1
:104500000840FFF7C7BF00BF00000240F46300206F
:1045100008B5084B1968890901F03D018A019A60C4
:10452000054AD3680BB110699847BDE80840FFF70A
:10453000B1BF00BF00000240F463002008B5084B83
:104540001968090C01F03D010A049A60054A536993
:104550000BB190699847BDE80840FFF79BBF00BFCB
:1045600000000240F463002008B5084B1968890D6B
:1045700001F03D018A059A60054AD3690BB1106AC2
:104580009847BDE80840FFF785BF00BF0000024024
:10459000F463002008B5074B074A596801F03D0154
:1045A000D960536A0BB1906A9847BDE80840FFF79D
:1045B00071BF00BF00000240F463002008B5084B43
:1045C0005968890901F03D018A01DA60054AD36A18
:1045D0000BB1106B9847BDE80840FFF75BBF00BF09
:1045E00000000240F463002008B5084B5968090C2C
:1045F00001F03D010A04DA60054A536B0BB1906B80
:104600009847BDE80840FFF745BF00BF00000240E3
:10461000F463002008B5084B5968890D01F03D018D
:104620008A05DA60054AD36B0BB1106C9847BDE878
:104630000840FFF72FBF00BF00000240F4630020D6
:1046400008B5074B074A196801F03D019960536CA2
:104650000BB1906C9847BDE80840FFF71BBF00BF47
:1046600000040240F463002008B5084B196889096A
:1046700001F03D018A019A60054AD36C0BB1106DBF
:104680009847BDE80840FFF705BF00BF000402409F
:10469000F463002008B5084B1968090C01F03D01CE
:1046A0000A049A60054A536D0BB1906D9847BDE8B6
:1046B0000840FFF7EFBE00BF00040240F463002093
:1046C00008B5084B1968890D01F03D018A059A600B
:1046D000054AD36D0BB1106E9847BDE80840FFF74F
:1046E000D9BE00BF00040240F463002008B5074BA8
:1046F000074A596801F03D01D960536E0BB1906EC5
:104700009847BDE80840FFF7C5BE00BF000402405F
:10471000F463002008B5084B5968890901F03D0190
:104720008A01DA60054AD36E0BB1106F9847BDE875
:104730000840FFF7AFBE00BF00040240F463002052
:1047400008B5084B5968090C01F03D010A04DA600C
:10475000054A536F0BB1906F9847BDE80840FFF7CB
:1047600099BE00BF00040240F463002008B5084B66
:104770005968890D01F03D018A05DA60054AD36F59
:1047800013B1D2F880009847BDE80840FFF782BE19
:1047900000040240F463002000230C4910B51A46BF
:1047A0000B4C0B6054F82300026001EB4300043310
:1047B0004260402BF6D1074A4FF0FF339360D3603D
:1047C000C2F80834C2F80C3410BD00BFF4630020F6
:1047D00010810008000002400F28F8B510D91028F9
:1047E00010D0112811D0122808D10F240720DFF88B
:1047F000C8E00126DEF80050A04208D9002653E0A8
:104800000446F4E70F240020F1E70724FBE706FA4B
:1048100000F73D424AD1264C4FEA001C3D4304EBD1
:1048200000160EEBC000CEF80050C0E90123FBB229
:1048300073B12048D0F8D83043F00103C0F8D83025
:10484000D0F8003143F00103C0F80031D0F8003156
:1048500017F47F4F0ED01748D0F8D83043F002033A
:10486000C0F8D830D0F8003143F00203C0F800316E
:10487000D0F8003154F80C00036823F01F030360E4
:10488000056815F00105FBD104EB0C033D2493F8FA
:104890000CC05F6804FA0CF43C602124056044619C
:1048A00012B1987B00F066F93046F8BD0130A3E7FD
:1048B0001081000800440258F463002010B5302431
:1048C00084F31188FFF788FF002383F3118810BD5C
:1048D00010B50446807B00F063F901231549627B23
:1048E00003FA02F20B6823EA0203DAB20B6072B930
:1048F000114AD2F8D81021F00101C2F8D810D2F82C
:10490000001121F00101C2F80011D2F8002113F4C6
:104910007F4F0ED1084BD3F8D82022F00202C3F803
:10492000D820D3F8002122F00202C3F80021D3F8E6
:10493000003110BDF46300200044025808B5302354
:1049400083F31188FFF7C4FF002383F3118808BDA8
:10495000026843681143016003B1184770470000C3
:10496000024A136843F0C0031360704700780040A8
:1049700013B50E4C204600F0BDFA04F114000023DC
:104980004FF400720A49009400F07AF9094B4FF491
:104990000072094904F13800009400F0F3F9074A65
:1049A000074BC4E9172302B010BD00BF7864002094
:1049B000E464002061490008E466002000780040BB
:1049C00000E1F505037C30B5244C002918BF0C46E6
:1049D000012B11D1224B98420ED1224BD3F8E82063
:1049E00042F08042C3F8E820D3F8102142F0804220
:1049F000C3F81021D3F810312268036EC16D03EBA8
:104A000052038466B3FBF2F36268150442BF23F0DD
:104A1000070503F0070343EA4503CB60A36843F0AF
:104A200040034B60E36843F001038B6042F49673EC
:104A300043F001030B604FF0FF330B62510505D5C6
:104A400012F0102205D0B2F1805F04D080F86430FB
:104A500030BD7F23FAE73F23F8E700BF108200084C
:104A600078640020004402582DE9F047C66D0546E1
:104A70003768F469210734621AD014F0080118BFAE
:104A80004FF48071E20748BF41F02001A3074FF0C7
:104A9000300348BF41F04001600748BF41F080014A
:104AA00083F31188281DFFF753FF002383F3118838
:104AB000E2050AD5302383F311884FF48061281D65
:104AC000FFF746FF002383F311884FF030094FF0C2
:104AD000000A14F0200838D13B0616D54FF03009F3
:104AE00005F1380A200610D589F31188504600F0E8
:104AF0007DF9002836DA0821281DFFF729FF27F065
:104B000080033360002383F31188790614D562068D
:104B100012D5302383F31188D5E913239A4208D1A3
:104B20002B6C33B127F040071021281DFFF710FF31
:104B30003760002383F31188E30618D5AA6E136942
:104B4000ABB15069BDE8F047184789F31188736A23
:104B5000284695F86410194000F0E6F98AF31188A8
:104B6000F469B6E7B06288F31188F469BAE7BDE882
:104B7000F0870000090100F16043012203F5614361
:104B8000C9B283F8001300F01F039A4043099B0049
:104B900003F1604303F56143C3F880211A60704755
:104BA00000F01F0301229A40430900F160409B007E
:104BB00000F5614003F1604303F56143C3F88020D1
:104BC000C3F88021002380F800337047F8B51546FC
:104BD000826804460B46AA4200D28568A16926690C
:104BE000761AB5420BD218462A46FCF7D3FEA369C3
:104BF0002B44A3612846A3685B1BA360F8BD0CD9B6
:104C0000AF1B18463246FCF7C5FE3A46E168304411
:104C1000FCF7C0FEE3683B44EBE718462A46FCF786
:104C2000B9FEE368E5E7000083689342F7B5044600
:104C3000154600D28568D4E90460361AB5420BD215
:104C40002A46FCF7A7FE63692B4463612846A368E4
:104C50005B1BA36003B0F0BD0DD93246AF1B0191C1
:104C6000FCF798FE01993A46E0683144FCF792FE61
:104C7000E3683B44E9E72A46FCF78CFEE368E4E797
:104C800010B50A440024C361029B8460C1600261C4
:104C90000362C0E90000C0E9051110BD08B5D0E904
:104CA0000532934201D1826882B982680132826002
:104CB0005A1C426119700021D0E904329A4224BF83
:104CC000C368436100F0C0FE002008BD4FF0FF3014
:104CD000FBE7000070B5302304460E4683F31188CD
:104CE000A568A5B1A368A269013BA360531CA36199
:104CF00015782269934224BFE368A361E3690BB18D
:104D000020469847002383F31188284607E0314660
:104D1000204600F089FE0028E2DA85F3118870BD94
:104D20002DE9F74F04460E4617469846D0F81C90DA
:104D30004FF0300A8AF311884FF0000B154665B129
:104D40002A4631462046FFF741FF034660B94146F7
:104D5000204600F069FE0028F1D0002383F311887B
:104D6000781B03B0BDE8F08FB9F1000F03D00190BC
:104D70002046C847019B8BF31188ED1A1E448AF325
:104D80001188DCE7C160C361009B82600362C0E9F7
:104D900005111144C0E9000001617047F8B50446EF
:104DA0000D461646302383F31188A768A7B1A36880
:104DB000013BA36063695A1C62611D70D4E904322F
:104DC0009A4224BFE3686361E3690BB120469847C8
:104DD000002080F3118807E03146204600F024FED1
:104DE0000028E2DA87F31188F8BD0000D0E9052336
:104DF00010B59A4201D182687AB9826800210132E5
:104E000082605A1C82611C7803699A4224BFC3687D
:104E1000836100F019FE204610BD4FF0FF30FBE724
:104E20002DE9F74F04460E4617469846D0F81C90D9
:104E30004FF0300A8AF311884FF0000B154665B128
:104E40002A4631462046FFF7EFFE034660B9414649
:104E5000204600F0E9FD0028F1D0002383F31188FB
:104E6000781B03B0BDE8F08FB9F1000F03D00190BB
:104E70002046C847019B8BF31188ED1A1E448AF324
:104E80001188DCE7026843681143016003B11847E9
:104E9000704700001430FFF743BF00004FF0FF33AE
:104EA0001430FFF73DBF00003830FFF7B9BF0000F6
:104EB0004FF0FF333830FFF7B3BF00001430FFF777
:104EC00009BF00004FF0FF311430FFF703BF0000AF
:104ED0003830FFF763BF00004FF0FF323830FFF784
:104EE0005DBF0000012914BF6FF013000020704760
:104EF000FFF73EBD044B036000234360C0E902336B
:104F000001230374704700BF2882000810B53023C6
:104F1000044683F31188FFF755FD02230020237414
:104F200080F3118810BD000038B5C36904460D46F2
:104F30001BB904210844FFF7A5FF294604F114001A
:104F4000FFF7ACFE002806DA201D4FF40061BDE833
:104F50003840FFF797BF38BD0268436811430160CE
:104F600003B118477047000013B5406B00F580543B
:104F7000D4F8A4381A681178042914D1017C0229C4
:104F800011D11979012312898B4013420BD101A948
:104F90004C3002F0D9F9D4F8A4480246019B21799B
:104FA000206800F0DFF902B010BD0000143002F0FC
:104FB0005BB900004FF0FF33143002F055B9000028
:104FC0004C3002F02DBA00004FF0FF334C3002F0AD
:104FD00027BA0000143002F029B900004FF0FF3169
:104FE000143002F023B900004C3002F0F9B900008F
:104FF0004FF0FF324C3002F0F3B900000020704750
:1050000010B500F58054D4F8A4381A681178042932
:1050100017D1017C022914D15979012352898B407F
:1050200013420ED1143002F0BBF8024648B1D4F856
:10503000A4484FF4407361792068BDE8104000F047
:105040007FB910BD406BFFF7DBBF00007047000069
:105050007FB5124B01250426044603600023057426
:1050600000F1840243602946C0E902330C4B0290F0
:10507000143001934FF44073009602F06DF8094B21
:1050800004F69442294604F14C000294CDE90063F1
:105090004FF4407302F034F904B070BD5082000840
:1050A00045500008694F00080A68302383F31188CF
:1050B0000B790B3342F823004B79133342F823006A
:1050C0008B7913B10B3342F8230000F58053C3F8FA
:1050D000A41802230374002080F311887047000095
:1050E00038B5037F044613B190F85430ABB90125AD
:1050F000201D0221FFF730FF04F114006FF00101C1
:10510000257700F0ADFC04F14C0084F854506FF0AA
:105110000101BDE8384000F0A3BC38BD10B5012145
:1051200004460430FFF718FF0023237784F8543037
:1051300010BD000038B504460025143002F024F8F4
:1051400004F14C00257702F0F3F8201D84F8545048
:105150000121FFF701FF2046BDE83840FFF750BFAF
:1051600090F8803003F06003202B06D190F8812066
:105170000023212A03D81F2A06D800207047222A9C
:10518000FBD1C0E91D3303E0034A4267072282676F
:10519000C3670120704700BF3C23002037B500F5EE
:1051A0008055D5F8A4381A68117804291AD1017CE1
:1051B000022917D11979012312898B40134211D189
:1051C00000F14C04204602F073F958B101A92046C1
:1051D00002F0BAF8D5F8A4480246019B217920686C
:1051E00000F0C0F803B030BD01F10B03F0B550F88A
:1051F000236085B004460D46FEB1302383F3118849
:1052000004EB8507301D0821FFF7A6FEFB6806F1B9
:105210004C005B691B681BB1019002F0A3F8019878
:1052200003A902F091F8024648B1039B29462046A3
:1052300000F098F8002383F3118805B0F0BDFB68F7
:105240005A691268002AF5D01B8A013B1340F1D13C
:1052500004F18002EAE70000133138B550F821402C
:10526000ECB1302383F3118804F58053D3F8A428DC
:105270001368527903EB8203DB689B695D6845B173
:1052800004216018FFF768FE294604F1140001F0BC
:1052900091FF2046FFF7B4FE002383F3118838BD49
:1052A0007047000001F05EBA01234022002110B5D2
:1052B000044600F8303BFCF793FB0023C4E90133BC
:1052C00010BD000010B53023044683F3118824225A
:1052D000416000210C30FCF783FB204601F064FAAA
:1052E00002230020237080F3118810BD70B500EBFD
:1052F0008103054650690E461446DA6018B1102243
:105300000021FCF76DFBA06918B110220021FCF709
:1053100067FB31462846BDE8704001F04BBB0000FA
:1053200083682022002103F0011310B50446836036
:105330001030FCF755FB2046BDE8104001F0C6BB1D
:10534000F0B4012500EB810447898D40E4683D43BA
:10535000A469458123600023A2606360F0BC01F072
:10536000E3BB0000F0B4012500EB810407898D4008
:10537000E4683D436469058123600023A2606360A3
:10538000F0BC01F059BC000070B5022300250446B2
:10539000242203702946C0F888500C3040F8045C81
:1053A000FCF71EFB204684F8705001F097FA636802
:1053B0001B6823B129462046BDE87040184770BDE0
:1053C0000378052B10B504460AD080F88C300523ED
:1053D000037043681B680BB1042198470023A36046
:1053E00010BD00000178052906D190F88C20436893
:1053F00002701B6803B118477047000070B590F841
:105400007030044613B1002380F8703004F180023C
:10541000204601F07FFB63689B68B3B994F8803045
:1054200013F0600535D00021204601F071FE002107
:10543000204601F061FE63681B6813B10621204617
:105440009847062384F8703070BD2046984700289E
:10545000E4D0B4F88630A26F9A4288BFA36794F96B
:105460008030A56F002B4FF0300380F20381002DB8
:1054700000F0F280092284F8702083F31188002163
:105480002046D4E91D23FFF76DFF002383F3118825
:10549000DAE794F8812003F07F0343EA022340F225
:1054A0000232934200F0C58021D8B3F5807F48D006
:1054B0000DD8012B3FD0022B00F09380002BB2D1EE
:1054C00004F1880262670222A267E367C1E7B3F5CD
:1054D000817F00F09B80B3F5407FA4D194F88230A7
:1054E000012BA0D1B4F8883043F0020332E0B3F5C9
:1054F000006F4DD017D8B3F5A06F31D0A3F5C063BE
:10550000012B90D86368204694F882205E6894F856
:105510008310B4F88430B047002884D043686367B0
:105520000368A3671AE0B3F5106F36D040F6024265
:1055300093427FF478AF5C4B63670223A367002339
:10554000C3E794F88230012B7FF46DAFB4F8883054
:1055500023F00203A4F88830C4E91D55E56778E715
:10556000B4F88030B3F5A06F0ED194F882302046A5
:1055700084F88A3001F010FA63681B6813B10121C6
:1055800020469847032323700023C4E91D339CE77A
:1055900004F18B0363670123C3E72378042B10D145
:1055A000302383F311882046FFF7BAFE85F3118874
:1055B0000321636884F88B5021701B680BB120466F
:1055C000984794F88230002BDED084F88B30042387
:1055D000237063681B68002BD6D0022120469847B1
:1055E000D2E794F8843020461D0603F00F010AD557
:1055F00001F082FA012804D002287FF414AF2B4B6B
:105600009AE72B4B98E701F069FAF3E794F88230B8
:10561000002B7FF408AF94F8843013F00F01B3D05F
:105620001A06204602D501F08BFDADE701F07CFDA6
:10563000AAE794F88230002B7FF4F5AE94F884301A
:1056400013F00F01A0D01B06204602D501F060FD2B
:105650009AE701F051FD97E7142284F8702083F354
:1056600011882B462A4629462046FFF769FE85F316
:105670001188E9E65DB1152284F8702083F3118862
:1056800000212046D4E91D23FFF75AFEFDE60B2238
:1056900084F8702083F311882B462A462946204639
:1056A000FFF760FEE3E700BF808200087882000811
:1056B0007C82000838B590F870300446002B3ED04C
:1056C000063BDAB20F2A34D80F2B32D8DFE803F0CA
:1056D00037313108223231313131313131313737DF
:1056E000856FB0F886309D4214D2C3681B8AB5FB23
:1056F000F3F203FB12556DB9302383F311882B4667
:105700002A462946FFF72EFE85F311880A2384F8DE
:1057100070300EE0142384F87030302383F3118846
:10572000002320461A461946FFF70AFE002383F39A
:10573000118838BDC36F03B198470023E7E7002104
:10574000204601F0E5FC0021204601F0D5FC63680D
:105750001B6813B10621204698470623D7E70000AF
:1057600010B590F870300446142B29D017D8062BAA
:1057700005D001D81BB110BD093B022BFBD800217D
:10578000204601F0C5FC0021204601F0B5FC63680D
:105790001B6813B1062120469847062319E0152BF4
:1057A000E9D10B2380F87030302383F31188002374
:1057B0001A461946FFF7D6FD002383F31188DAE76E
:1057C000C3689B695B68002BD5D1C36F03B1984751
:1057D000002384F87030CEE70023826803750369E4
:1057E0001B6899689142FBD25A680360426010605E
:1057F0005860704700238268037503691B689968C5
:105800009142FBD85A68036042601060586070474C
:1058100008B50846302383F311880A7D0023052A42
:1058200006D8DFE802F00B050503120E826913604B
:105830004FF0FF338361FFF7CFFF002383F311881D
:1058400008BD8269936801339360D0E90032136028
:105850005A60EDE7FFF7C0BF054BD96808751868B7
:10586000026853601A600122D8600275FAF7D2BD4F
:10587000E86800200C4B30B5DD684B1C87B004464F
:105880000FD02B46094A684600F07EF92046FFF704
:10589000E3FF009B13B1684600F080F9A86907B0E8
:1058A00030BDFFF7D9FFF9E7E8680020115800087C
:1058B00038B50C4D04468161EB6881689A68914265
:1058C00003D8BDE83840FFF787BF1846FFF792FFBF
:1058D00001230146EC6020462375BDE83840FAF705
:1058E00099BD00BFE8680020044B1A68DB68906827
:1058F0009B68984294BF002001207047E868002010
:10590000084B10B51C68D868226853601A600122E1
:10591000DC602275FFF76EFF01462046BDE81040AF
:10592000FAF778BDE868002038B50123084C002557
:105930002370656001F0F8FD01F01EFE0549064880
:1059400001F0F2FE0223237085F3118838BD00BFF9
:10595000506B002088820008E868002008B572B605
:10596000044B186500F026FD00F0E8FD024B032211
:105970001A70FEE7E8680020506B002000F044B980
:10598000034A516853685B1A9842FBD8704700BFBE
:10599000001000E08B600223086108468B8270478C
:1059A0008368A3F1840243F8142C026943F8442C61
:1059B000426943F8402C094A43F8242CC268A3F1F9
:1059C000200043F8182C022203F80C2C002203F8C4
:1059D0000B2C034A43F8102C704700BF2D0400081D
:1059E000E868002008B5FFF7DBFFBDE80840FFF7D7
:1059F00031BF0000024BDB6898610F20FFF72CBF1E
:105A0000E8680020302383F31188FFF7F3BF00001C
:105A100008B50146302383F311880820FFF72AFFD9
:105A2000002383F3118808BD064BDB6839B1426857
:105A300018605A60136043600420FFF71BBF4FF0EB
:105A4000FF307047E86800200368984206D01A6863
:105A50000260506018469961FFF7FCBE7047000075
:105A600038B504460D462068844200D138BD03682D
:105A700023605C608561FFF7EDFEF4E7036810B515
:105A80009C68A2420CD85C688A600B604C60216004
:105A9000596099688A1A9A604FF0FF33836010BD8D
:105AA000121B1B68ECE700000A2938BF0A2170B5F9
:105AB00004460D460A26601901F030FD01F018FD7C
:105AC000041BA54203D8751C04462E46F3E70A2E94
:105AD00004D90120BDE8704001F066BE70BD000031
:105AE000F8B5144B0D460A2A4FF00A07D96103F1A5
:105AF0001001826038BF0A224160196914460160B2
:105B000048601861A81801F0F9FC01F0F1FC431B92
:105B10000646A34206D37C1C28192746354601F0C9
:105B2000FDFCF2E70A2F04D90120BDE8F84001F09E
:105B30003BBEF8BDE8680020F8B506460D4601F00A
:105B4000D7FC0F4A134653F8107F9F4206D12A46CE
:105B500001463046BDE8F840FFF7C2BFD169BB68D7
:105B6000441A2C1928BF2C46A34202D92946FFF714
:105B70009BFF224631460348BDE8F840FFF77EBF51
:105B8000E8680020F8680020C0E90323002310B46F
:105B90005DF8044B4361FFF7CFBF000010B5194C0F
:105BA000236998420DD08168D0E9003213605A60B1
:105BB0009A680A449A60002303604FF0FF33A361A0
:105BC00010BD0268234643F8102F53600022026084
:105BD00022699A4203D1BDE8104001F099BC936854
:105BE00081680B44936001F083FC2269E16992684B
:105BF000441AA242E4D91144BDE81040091AFFF743
:105C000053BF00BFE86800202DE9F047DFF8BC80F3
:105C100008F110072C4ED8F8105001F069FCD8F8A4
:105C20001C40AA68031B9A423ED814444FF0000956
:105C3000D5E90032C8F81C4013605A60C5F80090DE
:105C4000D8F81030B34201D101F062FC89F3118819
:105C5000D5E9033128469847302383F311886B69CF
:105C6000002BD8D001F044FC6A69A0EB04098246FD
:105C70004A450DD2022001F097FD0022D8F81030DD
:105C8000B34208D151462846BDE8F047FFF728BF88
:105C9000121A2244F2E712EB09092946384638BFA6
:105CA0004A46FFF7EBFEB5E7D8F81030B34208D00C
:105CB0001444C8F81C00211AA960BDE8F047FFF79A
:105CC000F3BEBDE8F08700BFF8680020E868002058
:105CD00038B501F00DFC054AD2E90845031B181937
:105CE00045F10001C2E9080138BD00BFE8680020A5
:105CF00000207047FEE70000704700004FF0FF30C3
:105D00007047000002290CD0032904D0012907485C
:105D100018BF00207047032A05D8054800EBC200D1
:105D20007047044870470020704700BF6083000838
:105D30004C2300201483000870B59AB0054608462D
:105D4000144601A900F0C2F801A8FBF741FE431C6C
:105D50000022C6B25B001046C5E90034237003235D
:105D6000023404F8013C01ABD1B202348E4201D8B6
:105D70001AB070BD13F8011B013204F8010C04F8CD
:105D8000021CF1E708B5302383F311880348FFF7BD
:105D900005FA002383F3118808BD00BF586B00206B
:105DA00090F8803003F01F02012A07D190F881207B
:105DB0000B2A03D10023C0E91D3315E003F0600373
:105DC000202B08D1B0F884302BB990F88120212AFB
:105DD00003D81F2A04D8FFF7C3B9222AEBD0FAE769
:105DE000034A426707228267C3670120704700BFEA
:105DF0004323002007B5052917D8DFE801F019165D
:105E000003191920302383F31188104A01210190CE
:105E1000FFF76CFA019802210D4AFFF767FA0D4867
:105E2000FFF788F9002383F3118803B05DF804FBC2
:105E3000302383F311880748FFF752F9F2E7302344
:105E400083F311880348FFF769F9EBE7B482000890
:105E5000D8820008586B002038B50C4D0C4C2A46EF
:105E60000C4904F10800FFF767FF05F1CA0204F1CD
:105E700010000949FFF760FF05F5CA7204F1180028
:105E80000649BDE83840FFF757BF00BF3084002007
:105E90004C230020948200089E820008A9820008FA
:105EA00070B5044608460D46FBF792FDC6B2204683
:105EB000013403780BB9184670BD32462946FBF70A
:105EC00073FD0028F3D10120F6E700002DE9F0472B
:105ED00005460C46FBF77CFD2C49C6B22846FFF769
:105EE000DFFF08B11036F6B229492846FFF7D8FF80
:105EF00008B11036F6B2632E0BD8DFF89080DFF8C9
:105F00009090244FDFF898A02E7846B92670BDE80F
:105F1000F08729462046BDE8F04702F05DB8252EFF
:105F200030D1072241462846FBF73EFD80B91A4B87
:105F3000224603F1140153F8040B8B4242F8040B80
:105F4000F9D1198807359B78173411809370DBE7F6
:105F5000082249462846FBF727FD98B9A21C0F4B9B
:105F6000197802320909C95D02F8041C13F8011BF3
:105F700001F00F015345C95D02F8031CF0D118343C
:105F80000835C1E7013504F8016BBDE780830008DF
:105F9000A982000888830008F67F000800E8F11F46
:105FA0000CE8F11FBFF34F8F044B1A695107FCD166
:105FB000D3F810215207F8D1704700BF00200052DB
:105FC00008B50D4B1B78ABB9FFF7ECFF0B4BDA684C
:105FD000D10704D50A4A5A6002F188325A60D3F8D0
:105FE0000C21D20706D5064AC3F8042102F18832F3
:105FF000C3F8042108BD00BF8E8600200020005297
:106000002301674508B5114B1B78F3B9104B1A698A
:10601000510703D5DA6842F04002DA60D3F8102164
:10602000520705D5D3F80C2142F04002C3F80C21E9
:10603000FFF7B8FF064BDA6842F00102DA60D3F8E6
:106040000C2142F00102C3F80C2108BD8E8600200D
:10605000002000520F289ABF00F580604004002005
:10606000704700004FF40030704700001020704768
:106070000F2808B50BD8FFF7EDFF00F500330268D5
:10608000013204D104308342F9D1012008BD00203F
:10609000FCE700000F2838B505463FD8FFF782FF20
:1060A0001F4CFFF78DFF4FF0FF3307286361C4F8E3
:1060B00014311DD82361FFF775FF030243F0240359
:1060C000E360E36843F08003E36023695A07FCD48C
:1060D0002846FFF767FFFFF7BDFF4FF4003100F0E0
:1060E00009FA2846FFF78EFFBDE83840FFF7C0BF2A
:1060F000C4F81031FFF756FFA0F108031B0243F06C
:106100002403C4F80C31D4F80C3143F08003C4F8F4
:106110000C31D4F810315B07FBD4D9E7002038BD2F
:10612000002000522DE9F84F05460C46104645EA7E
:106130000203DE0602D00020BDE8F88F20F01F0029
:10614000DFF8BCB0DFF8BCA0FFF73AFF04EB0008B3
:10615000444503D10120FFF755FFEDE720222946F2
:10616000204601F007FF10B920352034F0E72B4618
:1061700005F120021F68791CDDD104339A42F9D160
:1061800005F178431B481C4EB3F5801F1B4B38BFED
:10619000184603F1F80332BFD946D1461E46FFF731
:1061A00001FF0760A5EB040C336804F11C0143F008
:1061B00002033360231FD9F8007017F00507FAD1E6
:1061C00053F8042F8B424CF80320F4D1BFF34F8FC8
:1061D000FFF7E8FE4FF0FF332022214603602846F8
:1061E000336823F00203336001F0C4FE0028BBD003
:1061F0003846B0E7142100520C20005214200052FF
:10620000102000521021005210B5084C237828B1FC
:106210001BB9FFF7D5FE0123237010BD002BFCD066
:106220002070BDE81040FFF7EDBE00BF8E86002055
:106230002DE9F04F0D4685B0814658B111F00D069D
:1062400014BF2022082211F00803019304D0431E3A
:1062500003426AD0002435E0002E37D009F11F0137
:1062600021F01F094FF00108324F05F00403DFF859
:10627000D0A005EA080BBBF1000F32D07869C00747
:106280002FD408F101080C37B8F1060FF3D19EB9ED
:10629000294D4946A819019201F090F904460028B9
:1062A0003AD11836019A782EF3D1494601F086F991
:1062B0000446002830D1019A4946204801F07EF971
:1062C000044668BB204605B0BDE8F08F0029C9D15F
:1062D00001462846029201F071F90446E0B9029A9B
:1062E000C0E713B178694107CBD5AC0702D578690F
:1062F0008007C6D5019911B178690107C1D5182069
:10630000494600FB08A0CDE9022301F057F90446F5
:10631000DDE902230028B4D04A460021204601E0EE
:106320004A460021FBF75CFBCCE70246002E95D1E4
:1063300098E700BF9C830008C0860020908600205C
:10634000A88600200121FFF773BF0000F8B5144DA7
:1063500001241827134E40F2FF3200210120FBF7E1
:106360003FFB07FB046001342A6955F80C1F01F05C
:1063700011F9062CF5D137254FF4C0542046FFF70C
:10638000E1FF014628B122460748BDE8F84001F088
:1063900001B9C4EBC404013D4FEAD404EED1F8BD09
:1063A0009C830008A88600209086002008B101F098
:1063B00077B9704738B5054D00240334696855F83E
:1063C0000C0B00F0A9F8122CF7D138BD9C83000803
:1063D00038B5EFF311859DB9EFF30584C4F30804D4
:1063E000302334B183F31188FFF772FC85F31188F1
:1063F00038BD83F31188FFF76BFC84F3118838BD37
:10640000BDE83840FFF764BC10B5FFF7E1FF104C62
:10641000C008104A002340EA4170C908A0FB04EC00
:10642000A0FB020E1CEB0000A1FB044CA1FB02121E
:106430005B41001943EB0C0011EB0E0142F100022D
:10644000411842F10000090941EA007010BD00BF87
:10645000CFF753E3A59BC4200244074BD2B210B53B
:10646000904200D110BD441C00B253F8200041F806
:10647000040BE0B2F4E700BF504000580E4B30B5BB
:106480001C6F240405D41C6F1C671C6F44F400446B
:106490001C670A4C02442368D2B243F48073236021
:1064A000074B904200D130BD441C51F8045B00B250
:1064B00043F82050E0B2F4E7004402580048025884
:1064C0005040005807B5012201A90020FFF7C4FF82
:1064D000019803B05DF804FB13B50446FFF7F2FF23
:1064E000A04205D0012201A900200194FFF7C6FFB8
:1064F00002B010BD0144BFF34F8F064B884204D356
:10650000BFF34F8FBFF36F8F7047C3F85C0220302B
:10651000F4E700BF00ED00E00144BFF34F8F064BEE
:10652000884204D3BFF34F8FBFF36F8F7047C3F818
:1065300070022030F4E700BF00ED00E0704700007B
:10654000074B45F255521A6003225A6040F2FF721F
:106550009A604CF6CC421A600122024B1A707047C6
:10656000004800583C870020034B1B781BB1034BAD
:106570004AF6AA221A6070473C870020004800585B
:10658000034B1A681AB9034AD2F8D0241A6070472C
:106590003887002000400258024B4FF48032C3F885
:1065A000D02470470040025808B5FFF7E9FF024BBE
:1065B0001868C0F3806008BD3887002070B5BFF34D
:1065C0004F8FBFF36F8F1A4A0021C2F85012BFF3EA
:1065D0004F8FBFF36F8F536943F400335361BFF3A1
:1065E0004F8FBFF36F8FC2F88410BFF34F8FD2F875
:1065F000803043F6E074C3F3C900C3F34E335B014C
:1066000003EA0406014646EA81750139C2F8605280
:10661000F9D2203B13F1200FF2D1BFF34F8F536912
:1066200043F480335361BFF34F8FBFF36F8F70BD5F
:1066300000ED00E0FEE70000214B2248224A70B541
:10664000904237D3214BC11EDA1C121A22F00302EA
:106650008B4238BF00220021FBF7C2F91C4A0023FD
:10666000C2F88430BFF34F8FD2F8803043F6E07425
:10667000C3F3C900C3F34E335B0103EA04060146CA
:1066800046EA81750139C2F86C52F9D2203B13F108
:10669000200FF2D1BFF34F8FBFF36F8FBFF34F8F38
:1066A000BFF36F8F0023C2F85032BFF34F8FBFF399
:1066B0006F8F70BD53F8041B40F8041BC0E700BF88
:1066C000CC850008308900203089002030890020E6
:1066D00000ED00E0074BD3F8D81021EA0001C3F821
:1066E000D810D3F8002122EA0002C3F80021D3F821
:1066F000003170470044025870B5D0E924430022AD
:106700004FF0FF359E6804EB42135101D3F80009A6
:10671000002805DAD3F8000940F08040C3F80009EA
:10672000D3F8000B002805DAD3F8000B40F08040C6
:10673000C3F8000B013263189642C3F80859C3F836
:10674000085BE0D24FF00113C4F81C3870BD0000A4
:10675000890141F02001016103699B06FCD41220EC
:10676000FFF70EB910B50A4C2046FEF79DFD094B08
:10677000C4F89030084BC4F89430084C2046FEF71B
:1067800093FD074BC4F89030064BC4F8943010BD0D
:10679000408700200000084008840008DC870020B3
:1067A000000004401484000870B503780546012BEE
:1067B0005CD1434BD0F89040984258D1414B0E21C8
:1067C0006520D3F8D82042F00062C3F8D820D3F86F
:1067D000002142F00062C3F80021D3F80021D3F871
:1067E000802042F00062C3F88020D3F8802022F09D
:1067F0000062C3F88020D3F88030FEF7BBF9324B3B
:10680000E360324BC4F800380023D5F89060C4F838
:10681000003EC02323604FF40413A3633369002BAD
:10682000FCDA01230C203361FFF7AAF83369DB0798
:10683000FCD41220FFF7A4F83369002BFCDA002601
:106840002846A660FFF758FF6B68C4F81068DB683D
:10685000C4F81468C4F81C6883BB1D4BA3614FF0D7
:10686000FF336361A36843F00103A36070BD194B5C
:106870009842C9D1134B4FF08060D3F8D82042F032
:106880000072C3F8D820D3F8002142F00072C3F898
:106890000021D3F80021D3F8802042F00072C3F821
:1068A0008020D3F8802022F00072C3F88020D3F833
:1068B0008030FFF70FFF0E214D209EE7064BCDE7FE
:1068C000408700200044025840140040030020028A
:1068D000003C30C0DC870020083C30C0F8B5D0F860
:1068E0009040054600214FF000662046FFF730FF3C
:1068F000D5F8941000234FF001128F684FF0FF304D
:10690000C4F83438C4F81C2804EB431201339F4206
:10691000C2F80069C2F8006BC2F80809C2F8080B97
:10692000F2D20B68D5F89020C5F898306362102336
:106930001361166916F01006FBD11220FFF720F83C
:10694000D4F8003823F4FE63C4F80038A36943F494
:10695000402343F01003A3610923C4F81038C4F89E
:1069600014380B4BEB604FF0C043C4F8103B094B9D
:10697000C4F8003BC4F81069C4F80039D5F8983061
:1069800003F1100243F48013C5F89820A362F8BD08
:10699000E483000840800010D0F8902090F88A101E
:1069A000D2F8003823F4FE6343EA0113C2F800383A
:1069B000704700002DE9F84300EB8103D0F89050B8
:1069C0000C468046DA680FFA81F94801166806F02D
:1069D0000306731E022B05EB41134FF0000194BF19
:1069E000B604384EC3F8101B4FF0010104F1100338
:1069F00098BF06F1805601FA03F3916998BF06F536
:106A0000004600293AD0578A04F15801374349011A
:106A10006F50D5F81C180B430021C5F81C382B18F3
:106A20000127C3F81019A7405369611E9BB3138A4D
:106A3000928B9B08012A88BF5343D8F89820981856
:106A400042EA034301F140022146C8F89800284673
:106A500005EB82025360FFF77BFE08EB8900C368F9
:106A60001B8A43EA845348341E4364012E51D5F8EF
:106A70001C381F43C5F81C78BDE8F88305EB49179F
:106A8000D7F8001B21F40041C7F8001BD5F81C18EB
:106A900021EA0303C0E704F13F030B4A28462146DD
:106AA00005EB83035A60FFF753FE05EB4910D0F85E
:106AB000003923F40043C0F80039D5F81C3823EA24
:106AC0000707D7E70080001000040002D0F89420E8
:106AD0001268C0F89820FFF70FBE00005831D0F8B8
:106AE000903049015B5813F4004004D013F4001FA8
:106AF0000CBF0220012070474831D0F89030490186
:106B00005B5813F4004004D013F4001F0CBF0220A4
:106B10000120704700EB8101CB68196A0B68136094
:106B20004B6853607047000000EB810330B5DD68AF
:106B3000AA691368D36019B9402B84BF402313603E
:106B40006B8A1468D0F890201C4402EB4110013C81
:106B500009B2B4FBF3F46343033323F0030343EAC2
:106B6000C44343F0C043C0F8103B2B6803F0030359
:106B7000012B0ED1D2F8083802EB411013F4807FBC
:106B8000D0F8003B14BF43F0805343F00053C0F8EB
:106B9000003B02EB4112D2F8003B43F00443C2F841
:106BA000003B30BD2DE9F041D0F8906005460C4621
:106BB00006EB4113D3F8087B3A07C3F8087B08D5E6
:106BC000D6F814381B0704D500EB8103DB685B683B
:106BD0009847FA071FD5D6F81438DB071BD505EB05
:106BE0008403D968CCB98B69488A5A68B2FBF0F63D
:106BF00000FB16228AB91868DA6890420DD2121A80
:106C0000C3E90024302383F3118821462846FFF787
:106C10008BFF84F31188BDE8F081012303FA04F2AD
:106C20006B8923EA02036B81CB68002BF3D02146EA
:106C30002846BDE8F041184700EB81034A0170B5D2
:106C4000DD68D0F890306C692668E66056BB1A445F
:106C50004FF40020C2F810092A6802F00302012A4A
:106C60000AB20ED1D3F8080803EB421410F4807F67
:106C7000D4F8000914BF40F0805040F00050C4F830
:106C8000000903EB4212D2F8000940F00440C2F8B8
:106C900000090122D3F8340802FA01F10143C3F8D4
:106CA000341870BD19B9402E84BF40202060206880
:106CB0001A442E8A8419013CB4FBF6F440EAC4401D
:106CC00040F00050C6E700002DE9F843D0F890608E
:106CD00005460C464F0106EB4113D3F8088918F01E
:106CE000010FC3F808891CD0D6F81038DB0718D577
:106CF00000EB8103D3F80CC0DCF81430D3F800E0CB
:106D0000DA68964530D2A2EB0E024FF000091A6005
:106D1000C3F80490302383F31188FFF78DFF89F3C4
:106D2000118818F0800F1DD0D6F834380126A640FF
:106D3000334217D005EB84030134D5F89050D3F8D3
:106D40000CC0E4B22F44DCF8142005EB0434D2F874
:106D500000E05168714514D3D5F8343823EA0606AB
:106D6000C5F83468BDE8F883012303FA01F203890A
:106D700023EA02030381DCF80830002BD1D09847C6
:106D8000CFE7AEEB0103BCF81000834228BF0346F7
:106D9000D7F8180980B2B3EB800FE3D89068A0F160
:106DA000040959F8048FC4F80080A0EB090898443E
:106DB000B8F1040FF5D818440B4490605360C8E74D
:106DC0002DE9F84FD0F8905004466E69AB691E402B
:106DD00016F480586E6103D0BDE8F84FFEF7D4BAC0
:106DE000002E12DAD5F8003E9B0705D0D5F8003EFC
:106DF00023F00303C5F8003ED5F80438204623F0FD
:106E00000103C5F80438FEF7EDFA370505D520462D
:106E1000FFF772FC2046FEF7D3FAB0040CD5D5F884
:106E2000083813F0060FEB6823F470530CBF43F4DB
:106E3000105343F4A053EB6031071BD56368DB6844
:106E40001BB9AB6923F00803AB612378052B0CD188
:106E5000D5F8003E9A0705D0D5F8003E23F003038D
:106E6000C5F8003E2046FEF7BDFA6368DB680BB14B
:106E700020469847F30200F1BA80B70226D5D4F82D
:106E8000909000274FF0010A09EB4712D2F8003B1F
:106E900003F44023B3F5802F11D1D2F8003B002B2F
:106EA0000DDA62890AFA07F322EA0303638104EB2D
:106EB0008703DB68DB6813B1394620469847013702
:106EC000D4F89430FFB29B689F42DDD9F00619D503
:106ED000D4F89000026AC2F30A1702F00F0302F41A
:106EE000F012B2F5802F00F0CA80B2F5402F09D120
:106EF00004EB8303002200F58050DB681B6A974295
:106F000040F0B0803003D5F8185835D5E90303D5E3
:106F100000212046FFF746FEAA0303D501212046A3
:106F2000FFF740FE6B0303D502212046FFF73AFE30
:106F30002F0303D503212046FFF734FEE80203D5D3
:106F400004212046FFF72EFEA90203D50521204685
:106F5000FFF728FE6A0203D506212046FFF722FE2E
:106F60002B0203D507212046FFF71CFEEF0103D5B6
:106F700008212046FFF716FE700340F1A780E907BD
:106F800003D500212046FFF79FFEAA0703D5012164
:106F90002046FFF799FE6B0703D502212046FFF735
:106FA00093FE2F0703D503212046FFF78DFEEE0643
:106FB00003D504212046FFF787FEA80603D5052147
:106FC0002046FFF781FE690603D506212046FFF71C
:106FD0007BFE2A0603D507212046FFF775FEEB0549
:106FE00074D520460821BDE8F84FFFF76DBED4F8F0
:106FF00090904FF0000B4FF0010AD4F894305FFAF4
:107000008BF79B689F423FF638AF09EB4713D3F8E5
:10701000002902F44022B2F5802F20D1D3F80029B4
:10702000002A1CDAD3F8002942F09042C3F8002964
:10703000D3F80029002AFBDB3946D4F89000FFF78B
:1070400087FB22890AFA07F322EA0303238104EB70
:107050008703DB689B6813B13946204698470BF1DC
:10706000010BCAE7910701D1D0F80080072A02F18D
:1070700001029CBF03F8018B4FEA18283FE704EB9D
:10708000830300F58050DA68D2F818C0DCF80820D5
:10709000DCE9001CA1EB0C0C00218F4208D1DB685D
:1070A0009B699A683A449A605A683A445A6029E758
:1070B00011F0030F01D1D0F800808C4501F10101DE
:1070C00084BF02F8018B4FEA1828E6E7BDE8F88F85
:1070D00008B50348FFF774FEBDE80840FDF7DAB9CC
:1070E0004087002008B50348FFF76AFEBDE8084066
:1070F000FDF7D0B9DC870020D0F8903003EB4111C8
:10710000D1F8003B43F40013C1F8003B7047000086
:10711000D0F8903003EB4111D1F8003943F400135B
:10712000C1F8003970470000D0F8903003EB4111EE
:10713000D1F8003B23F40013C1F8003B7047000076
:10714000D0F8903003EB4111D1F8003923F400134B
:10715000C1F800397047000030B50433039C017258
:10716000002104FB0325C160C0E90653049B0363AF
:10717000059BC0E90000C0E90422C0E90842C0E95B
:107180000A11436330BD00000022416AC260C0E9B9
:107190000411C0E90A226FF00101FEF761BC000092
:1071A000D0E90432934201D1C2680AB9181D704770
:1071B00000207047036919600021C2680132C26073
:1071C000C269134482699342036124BF436A036125
:1071D000FEF73ABC38B504460D46E3683BB1626938
:1071E0000020131D1268A3621344E36207E0237AB0
:1071F00033B929462046FEF717FC0028EDDA38BDE2
:107200006FF00100FBE70000C368C269013BC36087
:107210004369134482699342436124BF436A4361D3
:1072200000238362036B03B11847704770B53023A6
:10723000044683F31188866A3EB9FFF7CBFF054603
:1072400018B186F31188284670BDA36AE26A13F864
:10725000015B9342A36202D32046FFF7D5FF0023D0
:1072600083F31188EFE700002DE9F84F04460E463E
:10727000174698464FF0300989F311880025AA4631
:10728000D4F828B0BBF1000F09D141462046FFF7E2
:10729000A1FF20B18BF311882846BDE8F88FD4E90F
:1072A0000A12A7EB050B521A934528BF9346BBF170
:1072B000400F1BD9334601F1400251F8040B9142B3
:1072C00043F8040BF9D1A36A403640354033A3623A
:1072D000D4E90A239A4202D32046FFF795FF8AF3A6
:1072E0001188BD42D8D289F31188C9E730465A4681
:1072F000FAF750FBA36A5E445D445B44A362E7E790
:1073000010B5029C0433017203FB0421C460C0E980
:1073100006130023C0E90A33039B0363049BC0E9FF
:107320000000C0E90422C0E90842436310BD000028
:10733000026A6FF00101C260426AC0E904220022C1
:10734000C0E90A22FEF78CBBD0E904239A4201D19E
:10735000C26822B9184650F8043B0B6070470023FE
:107360001846FAE7C3680021C2690133C360436964
:10737000134482699342436124BF436A4361FEF729
:1073800063BB000038B504460D46E3683BB1236992
:1073900000201A1DA262E2691344E36207E0237A27
:1073A00033B929462046FEF73FFB0028EDDA38BD09
:1073B0006FF00100FBE7000003691960C268013A41
:1073C000C260C269134482699342036124BF436A65
:1073D000036100238362036B03B118477047000009
:1073E00070B530230D460446114683F31188866A32
:1073F0002EB9FFF7C7FF10B186F3118870BDA36ADD
:107400001D70A36AE26A01339342A36204D3E16967
:1074100020460439FFF7D0FF002080F31188EDE704
:107420002DE9F84F04460D46904699464FF0300A34
:107430008AF311880026B346A76A4FB94946204609
:10744000FFF7A0FF20B187F311883046BDE8F88F21
:10745000D4E90A073A1AA8EB0607974228BF17464D
:10746000402F1BD905F1400355F8042B9D4240F8ED
:10747000042BF9D1A36A40364033A362D4E90A232E
:107480009A4204D3E16920460439FFF795FF8BF354
:1074900011884645D9D28AF31188CDE729463A4664
:1074A000FAF778FAA36A3D443E443B44A362E5E719
:1074B000D0E904239A4217D1C3689BB1836A8BB188
:1074C000043B9B1A0ED01360C368013BC360C369C1
:1074D0001A4483699A42026124BF436A036100230C
:1074E00083620123184670470023FBE700F060BA6F
:1074F000014B586A704700BF000C0040034B00224C
:1075000058631A610222DA60704700BF000C004025
:10751000014B0022DA607047000C0040014B5863B9
:10752000704700BF000C0040024B034A1A60034A38
:107530005A607047908800203089002000000220A7
:10754000074B494210B55C68201A08401968821A36
:107550008A4203D3A24201D85A6010BD0020FCE742
:107560009088002008B5302383F31188FFF7E8FFE7
:10757000002383F3118808BD04480121044B0360F4
:107580000023C0E901330C3000F016B998880020C0
:1075900065750008CB1D083A23F00703591A521AE3
:1075A000012110B4D2080024C0E9004384600C30EB
:1075B0001C605A605DF8044B00F0FEB82DE9F84FEE
:1075C000364ECD1D0F46002818BF0646082A4FEA42
:1075D000D50538BF082206F10C08341D91464046F7
:1075E00000F006F909F10701C9F1000E22462468EE
:1075F0006CB9404600F006F93368CBB3082249461F
:10760000E8009847044698B340E9026730E004EB8D
:10761000010CD4F804A00CEA0E0C0AF10100ACF144
:10762000080304EBC0009842E0D9A0EB0C0CB5EBCA
:10763000EC0F4FEAEC0BD9D89C421CD204F10802A3
:10764000AB45A3EB02024FEAE202626009D9691C72
:10765000ED43206803EBC1025D44556043F83100FF
:1076600022601C465F60404644F8086B00F0CAF890
:107670002046BDE8F88FAA45216802D11160234653
:10768000EFE7013504EBC50344F8351003F10801B9
:10769000401AC01058601360F1E700BF98880020BE
:1076A000F8B550F8043C044650F8085CA0F1080610
:1076B00007332F1D0C35DB0840F8043C284600F04A
:1076C00097F83B469F421A6801D0B34228D20AB1CC
:1076D000964225D244F8082C54F8042C1E6001323E
:1076E00054F8081C06EBC200814206D148680244E7
:1076F00044F8042C0A6844F8082C5868411C03EB31
:10770000C1018E4207D154F8042C013202445A6060
:1077100054F8082C1A602846BDE8F84000F072B80A
:107720001346CFE7FEE7000070B51B4B002504466B
:1077300086B058600E4685620163FCF783FE04F153
:107740001003A560E562C4E904334FF0FF33C4E9D8
:107750000044C4E90635FFF7CBFE2B46024604F190
:1077600034012046C4E9082380230C4A2565FEF72E
:1077700011F901230A4AE0600092037568467268B5
:107780000192B268CDE90223064BCDE90435FEF73C
:1077900029F906B070BD00BF506B0020208400089E
:1077A0002584000825770008024AD36A1843D0626E
:1077B000704700BFE8680020C0E9000081607047A2
:1077C0008368013B002B10B583600CDA074BDC6843
:1077D0004368A061206063601C6044600520FEF780
:1077E0003BF8A06910BD0020FCE700BFE86800205E
:1077F00008B5302383F31188FFF7E2FF002383F3FA
:10780000118808BD08B5302383F3118883680133DC
:10781000002B836007DC036800211A680260506057
:107820001846FEF745F8002383F3118808BD0000D1
:107830004B6843608B688360CB68C3600B694361AE
:107840004B6903628B6943620B68036070470000F9
:1078500008B53C4B40F2FF713B48D3F888200A43FF
:10786000C3F88820D3F8882022F4FF6222F00702B0
:10787000C3F88820D3F88820D3F8E0200A43C3F85F
:10788000E020D3F808210A43C3F808212F4AD3F88F
:1078900008311146FFF7CCFF00F5806002F11C01B2
:1078A000FFF7C6FF00F5806002F13801FFF7C0FF67
:1078B00000F5806002F15401FFF7BAFF00F5806027
:1078C00002F17001FFF7B4FF00F5806002F18C0156
:1078D000FFF7AEFF00F5806002F1A801FFF7A8FFF7
:1078E00000F5806002F1C401FFF7A2FF00F580609F
:1078F00002F1E001FFF79CFF00F5806002F1FC015E
:10790000FFF796FF02F58C7100F58060FFF790FF9E
:1079100000F01AF90E4BD3F8902242F00102C3F89E
:107920009022D3F8942242F00102C3F89422052257
:10793000C3F898204FF06052C3F89C20054AC3F862
:10794000A02008BD00440258000002582C84000802
:1079500000ED00E01F00080308B500F0D7FAFDF7BE
:10796000E3FF104BD3F8DC2042F04002C3F8DC20E8
:10797000D3F8042122F04002C3F80421D3F80431E3
:10798000094B1A6842F008021A601A6842F00402B1
:107990001A60FEF7F5FDFEF7D9FCBDE80840FEF7DA
:1079A0005BBA00BF0044025800180248704700004C
:1079B000114BD3F8E82042F00802C3F8E820D3F8CE
:1079C000102142F00802C3F810210C4AD3F81031FC
:1079D000D36B43F00803D363C722094B9A624FF07D
:1079E000FF32DA6200229A615A63DA605A60012239
:1079F0005A611A60704700BF004402580010005CD2
:107A0000000C0040094A08B51169D3680B40D9B28F
:107A10009B076FEA0101116107D5302383F31188B9
:107A2000FDF7ACFF002383F3118808BD000C004074
:107A3000064BD3F8DC200243C3F8DC20D3F8042142
:107A40001043C3F80401D3F80431704700440258CE
:107A500008B53C4B4FF0FF31D3F8802062F0004274
:107A6000C3F88020D3F8802002F00042C3F88020C1
:107A7000D3F88020D3F88420C3F88410D3F884206E
:107A80000022C3F88420D3F88400D86F40F0FF4070
:107A900040F4FF0040F4DF4040F07F00D867D86F2B
:107AA00020F0FF4020F4FF0020F4DF4020F07F00B2
:107AB000D867D86FD3F888006FEA40506FEA50500B
:107AC000C3F88800D3F88800C0F30A00C3F8880020
:107AD000D3F88800D3F89000C3F89010D3F8900042
:107AE000C3F89020D3F89000D3F89400C3F8941012
:107AF000D3F89400C3F89420D3F89400D3F89800F6
:107B0000C3F89810D3F89800C3F89820D3F89800D9
:107B1000D3F88C00C3F88C10D3F88C00C3F88C20F9
:107B2000D3F88C00D3F89C00C3F89C10D3F89C10B9
:107B3000C3F89C20D3F89C30FCF72EFEBDE808402B
:107B400000F0B8B90044025808B50122534BC3F8FD
:107B50000821534BD3F8F42042F00202C3F8F4207A
:107B6000D3F81C2142F00202C3F81C210222D3F8F0
:107B70001C314C4BDA605A689104FCD54A4A1A60B1
:107B800001229A60494ADA6000221A614FF44042A9
:107B90009A61444B9A699204FCD51A6842F4807247
:107BA0001A603F4B1A6F12F4407F04D04FF48032BA
:107BB0001A6700221A671A6842F001021A60384BED
:107BC0001A685007FCD500221A611A6912F03802AF
:107BD000FBD1012119604FF0804159605A67344A46
:107BE000DA62344A1A611A6842F480321A602C4B05
:107BF0001A689103FCD51A6842F480521A601A6818
:107C00009204FCD52C4A2D499A6200225A631963CA
:107C100001F57C01DA6301F5E77199635A64284A3A
:107C20001A64284ADA621A6842F0A8521A601C4B99
:107C30001A6802F02852B2F1285FF9D148229A61FD
:107C40004FF48862DA6140221A621F4ADA641F4ADE
:107C50001A651F4A5A651F4A9A6532231E4A1360E5
:107C6000136803F00F03022BFAD10D4A136943F096
:107C700003031361136903F03803182BFAD14FF093
:107C80000050FFF7D5FE4FF08040FFF7D1FE4FF0D8
:107C90000040BDE80840FFF7CBBE00BF00800051A8
:107CA000004402580048025800C000F002000001E1
:107CB0000000FF0100889008322060006302090183
:107CC000470E0508DD0BBF01200000200000011059
:107CD0000910E00000010110002000524FF0B042F6
:107CE00008B5D2F8883003F00103C2F8883023B118
:107CF000044A13680BB150689847BDE80840FCF788
:107D0000C9BB00BFB08800204FF0B04208B5D2F820
:107D1000883003F00203C2F8883023B1044A936824
:107D20000BB1D0689847BDE80840FCF7B3BB00BF73
:107D3000B08800204FF0B04208B5D2F8883003F088
:107D40000403C2F8883023B1044A13690BB15069A7
:107D50009847BDE80840FCF79DBB00BFB0880020F5
:107D60004FF0B04208B5D2F8883003F00803C2F8EB
:107D7000883023B1044A93690BB1D0699847BDE8B4
:107D80000840FCF787BB00BFB08800204FF0B0422E
:107D900008B5D2F8883003F01003C2F8883023B158
:107DA000044A136A0BB1506A9847BDE80840FCF7D3
:107DB00071BB00BFB08800204FF0B04310B5D3F8BE
:107DC000884004F47872C3F88820A30604D5124AC8
:107DD000936A0BB1D06A9847600604D50E4A136BBC
:107DE0000BB1506B9847210604D50B4A936B0BB12E
:107DF000D06B9847E20504D5074A136C0BB1506C61
:107E00009847A30504D5044A936C0BB1D06C9847EE
:107E1000BDE81040FCF73EBBB08800204FF0B043F7
:107E200010B5D3F8884004F47C42C3F8882062057A
:107E300004D5164A136D0BB1506D9847230504D530
:107E4000124A936D0BB1D06D9847E00404D50F4AE8
:107E5000136E0BB1506E9847A10404D50B4A936E74
:107E60000BB1D06E9847620404D5084A136F0BB16A
:107E7000506F9847230404D5044A936F0BB1D06F19
:107E80009847BDE81040FCF705BB00BFB088002054
:107E900008B50348FCF7E8FDBDE80840FCF7FABA6E
:107EA0007864002008B5FFF7ADFDBDE80840FCF799
:107EB000F1BA0000062108B50846FCF75BFE062172
:107EC0000720FCF757FE06210820FCF753FE062189
:107ED0000920FCF74FFE06210A20FCF74BFE062185
:107EE0001720FCF747FE06212820FCF743FE092156
:107EF0007A20FCF73FFE07213220FCF73BFE0C21E5
:107F00005220BDE80840FCF735BE000008B5FFF779
:107F10009FFD00F00DF8FCF7EBFFFDF7C3F9FDF74F
:107F200095F8FFF743FDBDE80840FFF7DFBA000012
:107F30000023054A19460133102BC2E9001102F152
:107F40000802F8D1704700BFB08800200B460146F8
:107F5000184600F001B8000010B5054C13462CB1CE
:107F60000A4601460220AFF3008010BD2046FCE720
:107F70000000000010B501390244904201D10020F8
:107F800005E0037811F8014FA34201D0181B10BD82
:107F90000130F2E72DE9F041A3B1C91A1778014485
:107FA000044603F1FF3C8C42204601D9002009E041
:107FB0000578BD4204F10104F5D10CEB0405D61897
:107FC000A54201D1BDE8F08115F8018D16F801ED4B
:107FD000F045F5D0E7E70000034611F8012B03F860
:107FE000012B002AF9D170476F72672E6172647598
:107FF00070696C6F742E437562654F72616E676550
:108000002D7065726970682D686561767900000071
:1080100053544D333248373F3F3F0053544D333272
:10802000483733782F3732780053544D333248373E
:1080300034332F3735332F373530000001105A00D5
:1080400003105900012058000320560040A2E4F11B
:10805000646891060041A3E5F2656992070000009B
:1080600043414E464449666163653A204D657373EA
:108070006167652052414D204F766572666C6F775F
:10808000210000004261642043414E4966616365FE
:1080900020696E6465782E00000100000001FF0079
:1080A00000A0004000A4004000000000000000000C
:1080B000612B0008E9230008E93200085924000870
:1080C000652400087D280008DD250008212400081B
:1080D00025240008FD230008E523000839280008AE
:1080E0000924000851340008152400080D28000850
:1080F00001040E05054B02020E05054B04010E0599
:10810000054B05010B04044B080106030346000060
:1081100010000240080002400008024000000B006E
:1081200028000240080002400408024006010C003A
:1081300040000240080002400808024010020D0002
:1081400058000240080002400C08024016030E00CE
:10815000700002400C0002401008024000040F00B2
:10816000880002400C00024014080240060510007E
:10817000A00002400C000240180802401006110046
:10818000B80002400C0002401C08024016072F00F5
:108190001004024008040240200802400008380091
:1081A000280402400804024024080240060939005D
:1081B000400402400804024028080240100A3A0025
:1081C00058040240080402402C080240160B3B00F1
:1081D000700402400C04024030080240000C3C00D5
:1081E000880402400C04024034080240060D44009A
:1081F000A00402400C04024038080240100E450062
:10820000B80402400C0402403C080240160F46002D
:1082100000960000000000000000000000000000C8
:10822000000000000000000000000000B14E000847
:108230009D4E0008D94E0008C54E0008D14E0008DA
:10824000BD4E0008A94E0008954E0008E54E0008F6
:1082500000000000C94F0008B54F0008F14F0008AA
:10826000DD4F0008E94F0008D54F0008C14F000856
:10827000AD4F0008FD4F00080000000001000000A5
:108280000000000063300000848200084069002084
:10829000506B00204172647550696C6F7400254208
:1082A0004F415244252D424C002553455249414CE3
:1082B000250000000200000000000000E951000855
:1082C0005952000840004000008400201084002023
:1082D0000200000000000000030000000000000099
:1082E000A1520008000000001000000020840020BF
:1082F0000000000001000000000000004087002096
:1083000001010200F55D0008055D0008A15D00089F
:10831000855D0008430000001C830008090243003B
:10832000020100C03209040000010202010005241C
:1083300000100105240100010424020205240600A6
:1083400001070582030800FF09040100020A00007A
:1083500000070501024000000705810240000000FF
:1083600012000000688300081201100102000040A2
:10837000091241570002010203010000040309042D
:1083800025424F415244250030313233343536379F
:1083900038394142434445460000000000010020B6
:1083A00000FF010002000000000000300000040097
:1083B0000800000000000024000008000400000085
:1083C0000004000000FC0000020000000000043077
:1083D00000800000080000000000003800000100DC
:1083E0000100000000000000FD530008B556000821
:1083F00061570008400040007888002078880020FD
:10840000010000008888002080000000400100007A
:10841000080000000001000000100000080000003B
:108420006D61696E0069646C650000000000802A5F
:1084300000000000AAAAAAAA00000024FFFF000072
:108440000000000000A00A0000210002000000005F
:10845000AAAAAAAA00000000FFFF0000000000096D
:10846000000009001400005400000000AAAAAAAAF3
:1084700014000054FFFF0000000000000000000096
:108480000A40100000000000AAAA8AAA00401000BA
:10849000FFFF0000990000000000000000810200C2
:1084A00000000000AAAAAAAA00410100FFFF0000E4
:1084B0000000007007000000000000000000000045
:1084C000AAAAAAAA00000000FFFF00000000000006
:1084D000000000000000000000000000AAAAAAAAF4
:1084E00000000000FFFF000000000000000000008E
:1084F0000000000000000000AAAAAAAA00000000D4
:10850000FFFF00000000000000000000000000006D
:1085100000000000AAAAAAAA00000000FFFF0000B5
:10852000000000000000000000000000000000004B
:10853000AAAAAAAA00000000FFFF00000000000095
:10854000000000000000000000000000AAAAAAAA83
:1085500000000000FFFF000000000000000000001D
:10856000780500000000000000001E000000000070
:10857000FE2A0100D2040000FF000000586B00201A
:1085800078640020000000001080000883040000D0
:108590001B8000085004000029800008009600009D
:1085A0000000080096000000000800000400000021
:1085B0007C830008000000000000000000000000B4
:0C85C000000000000000000000000000AF
:00000001FF
